:100000003BC5000056C5000054C5000052C50000A5
:1000100050C500004EC500004CC500004AC5000098
:1000200048C5000046C500000C944E2D0C94362E99
:100030000C94940F3EC500003CC500003AC500007A
:1000400038C5000036C5000034C5000032C50000C8
:1000500030C500000C942A2D2CC500002AC50000D4
:1000600028C5000026C5000024C5000022C50000E8
:1000700020C500001EC500001CC500001AC50000F8
:1000800018C5000016C5000014C5000012C5000008
:1000900010C500000EC500000CC500000AC5000018
:1000A00008C5000006C5000004C5000005010904DC
:1000B000A101A1000501093009311601FE26FF0149
:1000C000950275108102C0C00660FF0961A1010997
:1000D00062150026FF00952075088102096315004E
:1000E00026FF00952075089102C005010906A101AF
:1000F000050719E029E7150025019508750181021A
:100100009501750881010507190029FF150026FFD3
:1001100000950675088100050819012905150025B7
:1001200001950575019102950175039101C000AF1C
:1001300000AE07087F0807003E5B4F5B3E003E6B4A
:100140004F6B3E001C3E7C3E1C00183C7E3C180061
:100150001C577D571C001C5E7F5E1C0000183C185D
:100160000000FFE7C3E7FF00001824180000FFE7C6
:10017000DBE7FF0030483A060E00262979292600E1
:10018000407F05050700407F05253F005A3CE73CBE
:100190005A007F3E1C1C0800081C1C3E7F001422D5
:1001A0007F2214005F5F005F5F0006097F017F0010
:1001B000006689956A0060606060600094A2FFA29A
:1001C000940008047E04080010207E201000080817
:1001D0002A1C0800081C2A0808001E101010100015
:1001E0000C1E0C1E0C0030383E383000060E3E0E41
:1001F000060000000000000000005F000000000793
:1002000000070000147F147F1400242A7F2A1200A4
:100210002313086462003649562050000008070383
:100220000000001C224100000041221C00002A1C8A
:100230007F1C2A0008083E0808000080703000007B
:10024000080808080800000060600000201008048A
:1002500002003E5149453E0000427F400000724985
:10026000494946002141494D33001814127F1000BE
:100270002745454539003C4A49493100412111098A
:100280000700364949493600464949291E00000001
:100290001400000000403400000000081422410057
:1002A0001414141414000041221408000201590906
:1002B00006003E415D594E007C1211127C007F49C0
:1002C000494936003E41414122007F4141413E00C3
:1002D0007F49494941007F09090901003E414151D7
:1002E00073007F0808087F0000417F410000204024
:1002F000413F01007F08142241007F404040400000
:100300007F021C027F007F0408107F003E414141B4
:100310003E007F09090906003E4151215E007F0928
:100320001929460026494949320003017F0103008B
:100330003F4040403F001F2040201F003F403840CA
:100340003F00631408146300030478040300615938
:10035000494D4300007F4141410002040810200044
:10036000004141417F00040201020400404040403E
:1003700040000003070800002054547840007F2804
:1003800044443800384444442800384444287F001A
:1003900038545454180000087E09020018A4A49C84
:1003A00078007F080404780000447D40000020406D
:1003B000403D00007F102844000000417F400000C5
:1003C0007C04780478007C080404780038444444B1
:1003D0003800FC182424180018242418FC007C0879
:1003E0000404080048545454240004043F442400E6
:1003F0003C4040207C001C2040201C003C40304001
:100400003C004428102844004C9090907C004464A8
:10041000544C440000083641000000007700000002
:100420000041360800000201020402003C26232697
:100430003C00000000000000404040F0F8F8FF38A9
:10044000FFF8F83FF8F8FF38FFF8F8F040404000B8
:10045000000000000080C0C0C0800000C0C080005C
:10046000000080C0C000C0C0000080C0C00000000C
:100470000000C0C0C0C0C000C0C00000000000003C
:10048000000000000000000000000000000000006C
:10049000000000000000000000000000000000005C
:1004A000000000000000000000000000000000004C
:1004B00000C0F0F8FC3E1E06010000007F414141F3
:1004C0007F007F4141417F000080C0E07E5B4F5B49
:1004D000FEC00000C000DCD7DEDEDED7DC00C000DE
:1004E000000000000000000000000000000000000C
:1004F0000000000000000000494949FFFFFFFFE045
:10050000DFBFBF00BFBFDFE0FFFFFFFF494949007A
:10051000000000001F3F6060E0BF1F007F7F071EDC
:10052000381E077F7F007F7F0E1F3B716000000039
:1005300000007F7F0C0C0C007E7E007F7E0303009A
:100540007F7E03037E7E03037F7E000F3E703C06AA
:100550003C703E0F00327B49493F7E007F7E0303A3
:10056000001E3F69696F26000000000000000000C7
:1005700000030F1F3F3C7870600000007F41414145
:100580007F007F4141417F00307B7F7830202030E9
:10059000787F3B0003000F7F0F0F0F7F0F000300DA
:1005A000000000000000000000000000000000004B
:1005B0000000000000000000010101070F0F7F0F85
:1005C0007F0F0F7E0F0F7F0F7F0F0F0701010100BD
:1005D0000000000000000000000101000000000019
:1005E000000000000000000000000000000000000B
:1005F00000000000000000000000000000000000FB
:1006000000000000000000000000000000000000EA
:1006100000000000000000000000000000000000DA
:1006200000000000000000000000000000000000CA
:1006300000000000000000000000000000000000BA
:1006400000000000000000000000000000000000AA
:10065000000000000000000000000000000000009A
:10066000000000000000000000000000000000008A
:10067000000000000000000000000000000000007A
:10068000000000000000000000000000000000006A
:100690000000000000007E0F00D4FFFFFFC7000035
:1006A000007800000000000000002A2B2800000055
:1006B0000000000000000000000000000029000011
:1006C00000002C1E3420212224342627252E362DEE
:1006D0003738271E1F202122232425263333362E88
:1006E00037381F0405060708090A0B0C0D0E0F10FA
:1006F0001112131415161718191A1B1C1D2F31303F
:10070000232D350405060708090A0B0C0D0E0F10E2
:100710001112131415161718191A1B1C1D2F31301E
:10072000354C09025B00030100A0FA090400000136
:100730000301010009211101000122440007058184
:10074000030800010904010002030000000921114F
:100750000100012222000705820320000107050392
:100760000320000109040200010300000009211117
:10077000010001221C00070584030800011201008A
:100780000200000008424105230100010203011C90
:10079000037600690061006C003A006600360034A0
:1007A000006300320062003300630000001A03524D
:1007B00000650070006C006900630061007A0065EC
:1007C0000072006F006E0000000603390052000046
:1007D0000004030904350029000D0010004F001724
:1007E0000020002100150028001B00E000E000E2CE
:1007F000005100E1002C00060009005000E1002338
:10080000001D00190052002B0061520C000500135E
:100810000000000000000000004F00000000000089
:10082000000000280000000000000000005100004F
:100830000000000000000050000000000000000068
:10084000005200000062520000000013000000008F
:1008500000000000004F0000000000000000002821
:100860000000000000000000005100000000000037
:1008700000000050000000000000000000520000D6
:100880000063520000000013002B782C783078337E
:10089000784F0000002578277823782800207800FA
:1008A00000000000005100037C267828782478504E
:1008B00000007C417E407E190052002178005200E9
:1008C000002278130000DA0281FFD9F1DB20A4A610
:1008D0002EAF00A0C0D30000A1C8D30000AED580C9
:1008E000A81F408D14200020004B6579636F64655C
:1008F000733A200020446973743A004469723A00E4
:100900004A6F79537469636B0057415344005741F0
:100910005344202B205368696674004D6F64653A18
:1009200020002000200044656661756C74005365EA
:100930007474696E6773004D6973630053686F6FF9
:10094000746572004C617965723A2000FD377A58FF
:100950005A000004E6D6B446020021011600000049
:10096000742FE5A3E0026200EC5D003D888986D328
:10097000DC0AE842C324925842588FD8E75CA0D2E0
:10098000616E26E888019A676C7887BC8D3709EA22
:100990002F54C1A53C7985897C2969B98F7792E567
:1009A000A65B868CA6AA91F9B95CB3C5C2123CA21B
:1009B00034DA88639433C51A9B63ED85DBE2AD2599
:1009C000B955023E39CABC49DFD0937191658EC7D3
:1009D0000C4A16371124AA533A3DF1D1EC32617F0B
:1009E000F99F216F9707AE524298410BA16EEEA678
:1009F000F70D43D1CBBA14DF35502A4D8615496D1A
:100A00007E3AD94D1CEC1AAE6A208011E9A236D983
:100A100043AE8531BA5B38C99DDB15A1FB593ECD8C
:100A20004DB516217CFE6F423A38CAF65306DBAC50
:100A3000E28F8C6D84AF8741D97CE0B1EEE9A2A250
:100A40000DB8D3E6BDCE2B4F4D74E03D4734EC9A44
:100A50006BC4B137772AE0001D6A4952C38D08760E
:100A600000018802E30400000257B588B1C467FBA7
:100A7000020000000004595A11241FBECFEFDAE033
:100A8000DEBFCDBF11E0A0E0B1E0E4E8F9E602C0CE
:100A900005900D92AC34B107D9F725E0ACE4B1E094
:100AA00001C01D92AA37B207E1F70E9493230C946C
:100AB0005534A6CA843018F05A9A5B9A0895982F34
:100AC000927080FD05C05A9A9115B9F35B9808950C
:100AD0005A98FACFCF93DF93C5E7D5E01B821A82ED
:100AE0001982188285E0FE01A0E7B5E001900D9221
:100AF0008A95E1F71C82DF91CF9108959C019A9528
:100B000081159F4118F5F32FF270EE27832F817026
:100B1000732F74706627532F5870442734FF0CC00E
:100B20008295807FEF2B09F08062672B09F080644B
:100B3000452B69F080680895EF2B09F08260672BE0
:100B400009F08460452B19F08860089580E00895CD
:100B5000CF93DF93EB01D2DFFE010995DF91CF91B7
:100B60000895982F92959F7024E0911102C020E083
:100B7000982F892F86958695811511F02E5F982FD5
:100B8000892F8695820F0895809325050895CF9328
:100B9000C82FE7DF809307048DDFC0932605CF9130
:100BA000089521E030E001C0220F8A95EAF7809194
:100BB0002605822BECCF21E030E0A90102C0440FD2
:100BC000551F8A95E2F7CA018095909126058923E1
:100BD000DECF292F963090F5853080F590E035E016
:100BE000239F800D911D1124282F277041E001C003
:100BF000440F2A95EAF723E0969587952A95E1F721
:100C0000FC01EE0FFF1FE80FF91FE850FC4F20E03A
:100C100030E070E05191DF01CB01022E02C09695C9
:100C200087950A94E2F7817081958527842385272B
:100C30008E932F5F3F4F2330310561F70895292FA1
:100C4000963078F5853068F590E035E0239F800D8B
:100C5000911D1124682F677023E0969587952A953A
:100C6000E1F7FC01EE0FFF1FE80FF91FE850FC4F02
:100C700040E050E080E0219130E0062E02C0369541
:100C800027950A94E2F721703327042E01C0220F22
:100C90000A94EAF7822B4F5F5F4F4330510559F7B3
:100CA000089580E008959091260521E030E0F90153
:100CB00001C0EE0F8A95EAF7D90102C0AA0FBB1F47
:100CC0006A95E2F7EA2B01C0220F4A95EAF7892FCD
:100CD0008E23E81303C0892F822B59CF2095822FB2
:100CE0008923FBCF80912E0590912D05981301C08B
:100CF00008958F5F8770FACF90912805809589239A
:100D000080932805282F2770211110C0891771F0B2
:100D100090916F0592FF0AC08695869586954BDF68
:100D20001092280510922A05109229050895909195
:100D30002305982B909323050895982F90958091E3
:100D40002305892380932305089580912205811529
:100D500031F01092220510922C0510922B05089567
:100D6000803E9105D9F1C8F48133910509F482C020
:100D700048F48932910509F472C08A32910509F468
:100D800080C0089589339105E9F082389105D1F04A
:100D90008533910509F45EC00895843E9105D9F12B
:100DA00048F4823E910539F1833E910549F181EE87
:100DB00090E00895863E9105C9F1873E910509F4BA
:100DC0003EC0089520916E052370211164C02091CA
:100DD0006F0523FF14C089E290E0089520916E050D
:100DE00020FD45C030916F0530FF09C024FD24C0AF
:100DF00083EE90E0089520916E0522FDF7CF0895CF
:100E000020916E0522FD44C030916F0530FD43C036
:100E100024FFF5CF11C020916F0521FFF0CF809105
:100E20006E0584FD09C087EE90E0089520916E055F
:100E300023FFE5CF24FFF7CF80E090E008952091D5
:100E40006E0523FD2BC030916F0531FFE1CF84EE9D
:100E500090E0089520916E0525FFD1CFBCCF209161
:100E60006E0525FD1EC020916F0523FFC8CF89E3C5
:100E700090E0089520916E0526FFC1CF8AE290E0B0
:100E8000089520916E0526FFBACF81E390E0089582
:100E900082EE90E0089580EE90E0089586EE90E076
:100EA000089585E390E0089590916E0592FF10C03B
:100EB00041E0282F2471243009F040E031E0282F50
:100EC0002871283009F030E0431711F02CE0822718
:100ED00093FF10C041E0282F2471243109F040E035
:100EE00031E0282F2871283109F030E0431711F044
:100EF0002CE0822730916F0530FF10C051E0282F81
:100F00002171213009F050E041E0282F287128306C
:100F100009F040E0541711F029E0822731FF10C09A
:100F200041E0282F2171213109F040E031E0282FE4
:100F30002871283109F030E0431711F029E08227A9
:100F400094FD877E08951F93CF93DF9309DFEC0113
:100F5000811522E5920708F044C0811540E5940709
:100F600008F0BAC0883E9105E0F4803E910560F437
:100F7000853A910570F4049738F481E0219709F0DF
:100F800080E0C82F50E0D52FCE01DF91CF911F9187
:100F900008958D5C9109D0654397B0F3C0E0D0E02F
:100FA000F3CFC11580E4D80798F4C11590E2D907B2
:100FB00008F0A8C0CE019A9581159F4178F78D2F32
:100FC00073DF182FCE019927CBDEEC01D12BDCCFBC
:100FD000CE019927C5DECC27DF70C82BD92BD06A6C
:100FE000D3CF803842E59407C8F5803652E595079F
:100FF00008F056C0C03482E5D807D0F4C03292E57C
:10100000D90708F046C08C2F8695869520E2829FEE
:10101000C0011124C37021E030E0A90102C0440FD7
:10102000551FCA95E2F7EA01C82BD92BDD68ACCF72
:101030008C2F86958695877050E2859FC00111247C
:10104000C37021E030E0A90102C0440F551FCA95CA
:10105000E2F7EA01C82BD92BDC6896CF803C52E539
:10106000950758F48F71C03AD24578F590E0982FE3
:101070008827EC01C46FD06A87CF805C9245809747
:1010800008F08CCFDC2FCC27CC27DF71C06FD06A63
:101090007BCFCF71D0E0DC2FCC27C16FD06A74CF6B
:1010A00086958695877020E2829FC0011124C370C7
:1010B00021E030E0A90102C0440F551FCA95E2F7B4
:1010C000EA01C82BD92BDA685FCFEEDEC82FD0E05B
:1010D000DC2FCC27D06258CF8F71E6DE93E0CC0FA7
:1010E000DD1F9A95E1F7CC27DF70282F30E084FFD1
:1010F00005C050E1859F900111243327C22BD32BCB
:10110000D06942CF8D2F8F71CFDE182FCE01992756
:1011100027DEEC01D12BDECF80E00895F894E82F94
:10112000E295EF70F0E041A18F7021E030E0B9016D
:1011300002C0660F771F8A95E2F7CB01962F909534
:10114000942391A392A1892B82A378940895811569
:101150002CE7920741F42091D7033091D803232B39
:1011600011F480E090E00895EBE9F4E080E090E095
:1011700065E072E248E252E22AE932E2778366836E
:101180005187408733872287978786870196709695
:101190008830910599F70895FC0184818623811197
:1011A0000AC082818115B9F06823908593FF05C03C
:1011B00081E061110FC080E00895282F22952F70E3
:1011C0008F70282B962F92959F706F70962B81E0D1
:1011D0002913F1CF089581E008950F931F93CF93C2
:1011E00001E010E0082E01C0000F0A94EAF7C09158
:1011F00021059C2F9023911115C09091280596955B
:1012000096959695891306C01092280510922A0586
:1012100010922905C6DCC027C0932105CF911F91EC
:101220000F910895C8DCF7CFFA01309709F00995BE
:101230000895E091EE03F091EF03309739F00190BB
:10124000F081E02D309711F00995089580E0089520
:101250009C01FC0132968FEF90E04191461751F0CE
:101260008F3F19F4411101C0892F9F5F9630A9F774
:101270008F3F09F40895280F311D87FD3A95F90134
:1012800062830895E0E5F1E09191891302C0DF01E6
:101290001E9291E0E635F907B9F7089580910301B0
:1012A00008952FB7F89460917B0170917C01809133
:1012B0007D0190917E012FBF0895CF92DF92EF9232
:1012C000FF92CF93DF93D82FC92FC0909504D09071
:1012D0009604E0909704F0909804E3DF6C197D0980
:1012E0008E099F09643F71408105910510F1D9DF96
:1012F0006B017C0182E390E0A0E0B0E0C0929B0132
:10130000D0929C01E0929D01F0929E018093970102
:1013100090939801A0939901B0939A01D09393046C
:10132000C0939404DF91CF91FF90EF90DF90CF9026
:10133000089584EF91E0A0E0B0E0E0CF87E797E781
:10134000909301088093000888E19AE00FB6F89422
:10135000A895809360000FBE90936000FFCF089522
:1013600008950895FC019B01809171019091720193
:101370008617970740F0672B29F48091E8008E7755
:101380008093E800C90140E0009741F4411106C094
:101390008091E80082FF2FC080E008952091D9035A
:1013A0002115A9F12530A9F12091E80023FD2DC0D8
:1013B0002091E80022FDECCF2091E80020FFE4CF4F
:1013C0003091F3002091F200009719F02830310598
:1013D00058F041E02830310509F040E02091E80064
:1013E0002E772093E800D0CF41914093F1000197F0
:1013F0002F5F3F4FE9CF8091D903811541F08530B0
:1014000041F08091E80083FFC3CF81E0089582E03E
:10141000089583E0089580916B0187FF13C0809148
:10142000E80082FF06C08091E8008B778093E80097
:1014300008958091D9038111F2CF08958091D90345
:101440008115D9F38091E80080FFF8CF8091E80002
:101450008E77ECCF2091E4003091E50095E6A9016C
:101460002091EC00822F817020FF06C08091E8005F
:1014700080FF06C080E008952091E80022FD1AC098
:101480008091D903811589F0853089F08091EB0036
:1014900085FD0FC02091E4003091E500421753070D
:1014A000F9F29A95E1F684E0089582E0089583E0E8
:1014B000089581E00895E8EDF0E080818E7F8083DB
:1014C0001092E2001092DA001092E100A0EEB0E07B
:1014D0008C9181608C9380818F77808319BCA7ED7C
:1014E000B0E08C918E7F8C9380818F7E8083109270
:1014F0006A010895E091EE03F091EF03309739F01F
:101500000284F385E02D309711F060E2099508958B
:10151000A0E0B0E0EEE8FAE00C9430336C0180918A
:101520000001909101018C159D0521F480916701C6
:10153000803269F1D0920101C092000180E2809373
:101540006701E12CF12C1092660106E611E0C0E083
:10155000D0E08AE0882E912CA12CB12CC701B601D5
:10156000A50194010E946D33605D603339F42097CA
:1015700029F0CD28CE28CF2809F460E2F801629343
:101580008F0169017A012196C530D10539F781E6CD
:1015900091E0CDB7DEB7ECE00C944C33982F9093EC
:1015A000E900891771F07091EC002091ED005091E5
:1015B000F00021FD09C09F5F973089F78093E90013
:1015C0000895762F242F50E03091EB003E7F30932A
:1015D000EB003091ED003D7F3093ED003091EB005A
:1015E00031603093EB007093EC002093ED0050934A
:1015F000F0002091EE0027FDDECF0895A0E0B0E0DE
:10160000E4E0FBE00C943433C8EDD0E088818F7EB9
:101610008883E7EDF0E080818160808384E082BF91
:1016200081E080936A0188818E7F888302EE10E0DA
:10163000F80110821092DA0081EEC82ED12CF6014A
:10164000108288818F7788838881806888838881E9
:101650008F7D888319BC1092D90310926901109272
:101660008F011092680190EEE92EF12CF701808134
:101670008B7F808388818160888342E060E080E0A6
:101680008DDFF60180818E7F8083F801808181600B
:101690008083808188608083F70180818E7F808352
:1016A000888180618883CDB7DEB7E8E00C94503341
:1016B000E0912E0590912D0527E0E91302C080E00E
:1016C0000895AE2FB0E02E9FF0011124E15DFA4F96
:1016D0003181361306C03081381303C0358134138D
:1016E00004C0FD013196E770E8CF81E008950F93C3
:1016F0001F93CF93DF938B01EA019091D90394302C
:1017000051F58093E9008FEF9091E80095FD06C0B8
:1017100095ED9A95F1F700008A95B1F78091E80070
:1017200085FF19C097DE811111C08091E80085FD09
:1017300006C08091E8008E778093E800F3CFF8012F
:1017400081918F018093F100219779F78091E800D2
:101750008E778093E800DF91CF911F910F910895CC
:10176000792F603229F440E250E0682F82E0BFCF49
:101770000895CF93DF93D82FC92F48E050E0682F0A
:10178000792F81E0B4DF88E0ED2FFC2FA3E7B1E0F3
:1017900001900D928A95E1F7DF91CF910895909194
:1017A0006F0592FB222720F9281771F080FB92F930
:1017B00090936F0560916E0570916F0584E090E0E5
:1017C0000E943A3482E098CA08951F93CF93DF9322
:1017D000962F122F632F8430D8F49630C8F44530FA
:1017E000B8F4C42FD0E0CC0FDD1F2AE0929FC00DCB
:1017F000D11D11249CE3899FC00DD11D1124CE0160
:1018000089960E942034612FCE018A960E9420344E
:10181000DF91CF911F9108950F931F93CF93DF9383
:10182000843030F5663020F5453010F5C42FD0E017
:10183000CC0FDD1F2AE0629FC00DD11D11243CE3B7
:10184000839FC00DD11D1124CE0189960E940434BE
:10185000082F10E0102F0027CE018A960E94043432
:101860009801282BC901DF91CF911F910F91089505
:1018700080E090E0F8CF462F672F2091EA03309167
:10188000EB03232B81F4703F39F4403F61F48091E6
:10189000E8039091E9030895763028F4453018F470
:1018A000843008F4B9CF80E090E00895A0E0B0E083
:1018B000ECE5FCE00C9435337C0100912605809129
:1018C0002505082BC3E0D0E010E0C8010C2E02C0B3
:1018D000959587950A94E2F780FD09C02197A8F7AE
:1018E000D12C8D2DCDB7DEB7E7E00C945133DC2E33
:1018F000B7018C2FC0DF27DB019781F3F2CF0F9365
:101900001F93CF93FC01858100811181811579F0AE
:10191000611569F0C801CADFC82F682FC80159D9FD
:10192000B8018C2FA8DFCF911F910F910895C801A6
:1019300086D9C82FF5CFCF93DF93D82FC92FB6DF25
:101940006D2F7C2F98DFFFDADF91CF910895FC0196
:101950008481811599F080819181EDDF282F929506
:101960009F70963099F060F4925F9F70923030F4DF
:10197000203FB1F038F481E0283E38F080E008954F
:101980009A5FF3CF81E0243FC9F7089591E0213FAA
:1019900009F090E081E0283E08F080E0892B08956E
:1019A00081E00895382F292FCB01A32FB22F873440
:1019B00022E09207A105B10520F487549E4F0C94B4
:1019C000043480E0089585E290E00E9404348E396A
:1019D00089F486E290E00E9404348F3559F487E25E
:1019E00090E00E94043491E08E3E09F090E0892F4F
:1019F0008170089580E0FCCFAAE0B0E0E2E0FDE075
:101A00000C942F33C090D703D090D80381E090E09E
:101A10009093D8038093D703812C912CE12C54010F
:101A2000F12C14C0F80125913591472D6F2D8E2D85
:101A3000CCDE0E5F1F4F739485E07812F3CF95E0F4
:101A4000A90EB11CF394E6E0FE1639F08501000FF3
:101A5000111F0B52184F712CE5CFE394FEE18F0E4E
:101A6000911C84E0E812DBCF1A8219821C821B824F
:101A70001E821D8218861F8288EC90E09A878987D3
:101A800009E111E0FE0131967F014AE050E0B80122
:101A9000C7010E943E34065F1F4F57010936F1E02F
:101AA0001F0799F789E0F70111928A95E9F78FEFFF
:101AB0009FEF9E838D8387E08A874AE050E0B801DC
:101AC000C5010E943E34065F1F4F093BF1E01F072E
:101AD000A1F7D092D803C092D7032A96EDE00C94D8
:101AE0004B33AAE0B0E0E7E7FDE00C94323308E1C5
:101AF00014E089E6E82EFF24F39497E0B92E2FE74F
:101B0000C22E21E0D22EAA24A3944AE050E0B701CD
:101B1000CE0101960E94F433F8013896DF018B2D37
:101B20001D928A95E9F789819A81D80111969C9333
:101B30008E938F8112968C9312978D8113968C932E
:101B40001397888514968C931497898515968C9392
:101B500015978B819C8117969C938E9316978A85F7
:101B600087FD04C01E96DC92CE921D9780FF02C0B6
:101B7000F801A08681FF07C0D80118969C9118979C
:101B8000926018969C9382FF04C0F801908594603F
:101B9000908783FF07C0D80118969C91189798608A
:101BA00018969C9384FF04C0F801908590619087FB
:101BB00085FF07C0D80118968C91189780621896F7
:101BC0008C93BAE0EB0EF11C015F1F4FE9EBEE16B0
:101BD000E1E0FE0609F099CF2A96EAE00C944E3334
:101BE000282FCB01283070F44AE0249F9001112463
:101BF000B901675E7E4F4AE050E00E94F43380E016
:101C000090E008958FEF9FEF0895AAE0B0E0EBE039
:101C1000FEE00C943A339C0197558115914068F48D
:101C2000BE016F5F7F4F822FDBDF892B31F4898507
:101C30009A852A96E2E00C94563388EC90E0F9CF2E
:101C4000AB0124E630E0BC0188E70E94AD2F9C0187
:101C500081E0232B09F080E008958091CB0381156A
:101C600061F08091CA03811541F062E070E080E389
:101C700091E0E6DF81111092CA0308958091CB03B1
:101C80008115E9F00EDBDC01CB01805A9541AF4FA5
:101C9000BF4F8093C6039093C703A093C803B0932C
:101CA000C9038091CA0381110AC062E070E08EE22C
:101CB00091E0C6DF811519F081E08093CA03089591
:101CC000A0E1B0E0E6E6FEE00C942C33FE01319694
:101CD00080E1DF011D928A95E9F705E210E099EBBA
:101CE000A92EBB24B39427E4422E22E0522E612C6D
:101CF000712C4F0173016201B1E14B165104610473
:101D000071041CF080E1C82ED12CA601B501C401DC
:101D10000E941134AC0CBD1C0D2C000CEE08FF0809
:101D20004C185D086E087F080150104019F7609646
:101D3000E0E10C9448336FEF85E290E00E9420349C
:101D40006FEF86E290E00E9420346FEF87E290E030
:101D50000E94203460E088E290E00E9420344CDE53
:101D6000AFDF6EE985E290E00E9420346FE586E205
:101D700090E00E9420346EEE87E290E00C942034D4
:101D8000CF93DF93682F81E06A3019F06D3029F42A
:101D900080E075D0DF91CF91089580919F0190915F
:101DA000A00126E0FC01ABE5B1E001900D922A957F
:101DB000E1F7603E08F458C026E0FC0111922A9534
:101DC000E9F7C0919F01D091A00146E050E0BE012B
:101DD0008BE591E00E94E0339E01225C3140892B2B
:101DE00041F1C90145E0969587954A95E1F741E0B3
:101DF00050E0BA0102C0660F771F8A95E2F7CB0167
:101E00006091C4037091C503862B972BB9016B5F5A
:101E10007F4FE5E076956795EA95E1F702C0440FBC
:101E2000551F6A95E2F7842B952B9093C5038093F9
:101E3000C4032A5F3F4F4091A101642F70E0C901A4
:101E40000E941633481B463010F4240F311D211513
:101E500072E0370710F020E030E02E533E4F309311
:101E6000A00120939F0196CFF6E06F9FB00111244F
:101E70006E5C7E4F46E050E00E94D733A2CFCF93F6
:101E8000382FE0919F01F091A001E25CF140209198
:101E9000A101622F70E0CF010E941633281B822F10
:101EA000311559F066E00E946133C82FC15010F41B
:101EB000CF91089580E264DFF9CF8E0F9F2F911D9F
:101EC000811522E0920710F080E090E08E539E4F43
:101ED0009093A00180939F01EBCFCF93DF93EC0110
:101EE000FE018491811103C0DF91CF91089548DFF5
:101EF0002196F6CFF2DF81E0C2CF0F931F93CF93ED
:101F0000DF93EC01FC0101900020E9F78F01015003
:101F10001109C017D10728F0DF91CF911F910F91C0
:101F2000089589912DDFF5CF1F921FB61F921124BE
:101F30008F939F93AF93BF9380918E01811113C0B4
:101F400080917B0190917C01A0917D01B0917E01F7
:101F50004196A11DB11D80937B0190937C01A093BC
:101F60007D01B0937E01BF91AF919F918F911F90A2
:101F70001FBE1F9018952FB7F89480917B01909108
:101F80007C01A0917D01B0917E012FBF0895CF9378
:101F9000DF93C091230580912705C82B80912205EE
:101FA0008115F1F0E8DF20912B0530912C05821B83
:101FB000930B8838934110F00E94A506D09122051A
:101FC00020E080E591E0FC013081019631112F5F26
:101FD00031E086359307B9F721110E94A506CD2B74
:101FE0008091170480958C2390911604892B8093FF
:101FF0004E0148E050E060EF73E08EE491E00E9413
:10200000E033892BB9F088E0EEE4F1E0A0EFB3E033
:1020100001900D928A95E1F7E091EE03F091EF03C4
:10202000309741F00280F381E02D309719F08EE473
:1020300091E00995DF91CF91089510922305E0E595
:10204000F1E086E0DF011D928A95E9F710922705FD
:102050009ECFF3DF2FEF84E39CE02150804090403F
:10206000E1F700C0000088E19AE00FB6F894A89567
:10207000809360000FBE90936000FFCFAAE2B0E0B3
:10208000E4E4F0E10C9439338BE691E0FC01019635
:102090002091F100208321E083379207B9F78091E6
:1020A0006C01893009F457C0C8F4823009F4B1C01A
:1020B000833009F481C0813081F18091E80083FF91
:1020C000E5C080916B0190916C019A3008F0DEC000
:1020D000E92FF0E0E259FB4C0C94AB338A3009F461
:1020E00088C08B3051F780916B01813231F780913C
:1020F0006F0190917001892B01F78091E800877F33
:102100008093E80088D981E090916D01911101C020
:1021100080E08093040191DFD0CF80916B01813A00
:1021200061F68091E800877F8093E80080916F01DD
:1021300090917001892B59F060E080E090E070E0B0
:1021400011D98091E8008B778093E800B6CF68E0E2
:1021500083E791E0F4CF80916B01813209F0ADCF3C
:1021600080916F0190917001892B09F0A6CF809129
:10217000E800877F8093E8008091E80082FF17C025
:102180009091F3008091F200029731F48091F10078
:10219000813011F0863021F48091F10080930301A9
:1021A0008091E8008B778093E80035D986CF8091C5
:1021B000D9038111E1CF81CF80916B01813A09F080
:1021C0007CCF80916F0190917001892B09F075CFC0
:1021D0008091E800877F8093E8008091E80080FF8D
:1021E000FCCF809104018093F1008091E8008E770C
:1021F000DACF80916B01813209F05FCF8091E800E6
:10220000877F8093E80007D980916E018093020157
:1022100054CF80916B01813A09F04FCF8091E80053
:10222000877F8093E8008091E80080FFFCCF809159
:102230000201D9CF803889F0823841F580916F0151
:102240008F70873018F58093E9008091EB0085FB53
:10225000882780F91092E90006C080918F01880FCD
:1022600090916801892B9091E800977F9093E80006
:102270008093F1001092F1008091E8008E7723C0E6
:10228000811116C080916D01813009F18091E800C3
:1022900083FF0AC08091E800877F8093E8008091E7
:1022A000EB0080628093EB00AA96E3E00C94553338
:1022B000823061F780916D01811581F01092E90003
:1022C0008091E800877F8093E800A5D8DFCF81E088
:1022D000933009F080E080938F01F0CF80916F01FF
:1022E0008F702FEF280F263088F68093E900209119
:1022F000EB0020FFE3CF933031F48091EB0080625C
:102300008093EB00DBCF9091EB0090619093EB001A
:1023100021E030E0A90102C0440F551F8A95E2F781
:102320004093EA001092EA008091EB008860E8CFC9
:102330008111ACCF10916D011F778091E3008078FF
:10234000812B8093E3008091E800877F8093E800F1
:1023500062D88091E80080FFFCCF8091E300806824
:102360008093E30083E0111101C082E08093D903E0
:102370008DCF8058823008F089CF80916D01909187
:102380006E018C3D53E0950799F583E08A838AE2DC
:1023900089834FB7F894DE01139620E03EE051E2C6
:1023A000E32FF0E050935700849120FF03C0829503
:1023B0008F703F5F8F708A30C8F0895C90E08D939A
:1023C0009D932F5F243161F74FBF8091E800877F95
:1023D0008093E8006AE270E0CE0101960E94B209A3
:1023E0008091E8008B778093E80050CF805DE6CF46
:1023F000292F33272330310509F44EC078F52130D9
:10240000310509F488C08BE590E0E2E2F7E0223084
:10241000310509F03BCF2091E800277F2093E800A9
:1024200020917101309172018217930708F49C0189
:1024300040E02115310509F073C0411171C0809150
:10244000E80082FDCDCF8091D903811549F2853016
:1024500039F28091E80083FFF2CFC2CF80916F0103
:10246000909170012132310509F446C022323105C4
:1024700009F00CCF8330910508F008CFFC01EE0F76
:10248000FF1FE45DFE4F0190F081E02D875D9E4FC0
:10249000DC018C9190E010C09C013327823021F147
:1024A0002330310568F4232BB9F4E1EDF7E0E49132
:1024B0008E2F90E0E1EDF7E0009709F4E7CEABCF87
:1024C0002330310509F0E2CEEFE8F7E0E4918E2FFA
:1024D00090E0EFE8F7E0F0CFE9ECF7E0E4918E2F41
:1024E00090E0E9ECF7E0E8CFEDEAF7E0E4918E2F39
:1024F00090E0EDEAF7E0E0CF8330910508F0C6CE3A
:10250000FC01EE0FFF1FEE5CFE4F0190F081E02D0D
:1025100089E090E080CF82E190E0EDE7F7E07BCFCB
:102520008091D903811509F45BCF853009F458CF28
:102530008091E80083FD54CF8091E80082FD7FCF39
:102540008091E80080FF75CF9091F3008091F200B8
:102550002115310519F08830910550F041E00897B8
:1025600009F040E08091E8008E778093E80061CF29
:1025700044914093F1003196215031090196E8CF02
:10258000803809F083CE8091E800877F8093E8004F
:10259000809169018093F1006FCE811177CE109107
:1025A0006D01123008F072CE8091E800877F809331
:1025B000E800109369010E940B0A1115F9F084E0FC
:1025C0008093D90342E061EC81E00E94CE0A42E2AE
:1025D00061EC82E00E94CE0A42E260EC83E00E945D
:1025E000CE0A42E061EC84E00E94CE0A8091D903D9
:1025F000843051F482E08093050148CE8091E3005D
:1026000087FDDDCF81E0DCCF81E0F5CFCF93C82F10
:10261000811599F08CEF8C0F813A88F4E0E5F1E0B8
:102620008191C817C9F081E0E635F807C9F76C2F2A
:102630008EE491E00E942809AADCCF91089580E2FF
:102640008C0F8830D0F7C77081E001C0880FCA9521
:10265000EAF70E949706F0CF8C2F0E94420997DC80
:10266000E6CFCF93DF93EC01805E9109089720F0CD
:1026700064E474E1209711F468E374E1CE010E94F0
:10268000A8058C2FC3DFDF91CF910895811539F014
:102690009CEF980F913A20F40E94420978CC08955B
:1026A00090E2980F9830D8F7877091E001C0990FA9
:1026B0008A95EAF7892F0E949D06F0CFCF93DF938A
:1026C000EC01E4DFCE01805E9109089720F06DE413
:1026D00074E1209711F46EE374E1CE010E94A80525
:1026E000DF91CF910895611519F0411102C0B9CF62
:1026F000E5CF08951F93CF93DF93182FEB0186DF6B
:10270000209731F4812FC2DFDF91CF911F9108957F
:102710008FE99FE00197F1F700C000002197F0CF0B
:10272000A0E0B0E0E6E9F3E10C943333EC018881FA
:10273000811509F1813009F045C08981813051F45A
:102740008A81239660E570E0893311F060E070E0E3
:10275000D1DFEDCF823021F48A81239657DFE7CF96
:10276000833021F48A81239691DFE1CF843041F0D8
:1027700022968111DCCFCDB7DEB7E9E00C944F3360
:102780008A81239620E030E09AE0682F6053770B2F
:10279000AB016A30710560F02115310551F3EFE9A5
:1027A000FFE03197F1F700C0000021503109F4CF6C
:1027B000929FB001939F700D11249A01260F371F2D
:1027C0008991E3CFE82FF0E0EE55F94FB490282F30
:1027D00026952695269530E0F901EE56F94FE490BE
:1027E0008770F12C082E02C0F594E7940A94E2F762
:1027F000E0FAEE24FF24E0F8F901EE57F94FC49017
:10280000D12C082E02C0D594C7940A94E2F7C0FADE
:10281000CC24DD24C0F8F901EE58F94F049110E002
:1028200002C0159507958A95E2F701701127E1140A
:10283000F10411F081EEEADEC114D10411F086EE4C
:10284000E5DE60E070E08B2D55DFC114D10411F09E
:1028500086EE1CDFE114F10411F081EE17DF0115A3
:10286000110521F060E070E08CE244DF21965FCF3B
:10287000811519F00E9497068ACB0895811519F0E9
:102880000E949D0684CB0895811531F09091270513
:10289000892B809327057BCB0895811539F080958E
:1028A0009091270589238093270571CB0895809106
:1028B0001204811521F082E2F0DF109212040895D3
:1028C000CF93DF93EC014A855B856E857F850E94FF
:1028D00014099B8190958091270589238093270572
:1028E0008C810E949D0653DB86E0FE0111928A9541
:1028F000E9F7DF91CF910895CF93DF93EC018D81BC
:1029000081FD13C082608D83809127059B81892B77
:10291000809327058C810E94970639DB488559856D
:102920006E857F85CE010E94140910921C051092BD
:102930001B058D8180FD02C0CE01C2DFDF91CF91EA
:1029400008951F93CF93DF93182FA0919104B09116
:102950009204109709F449C01092940410929304C1
:1029600010921704109216041696CD91DC911797C9
:10297000CE019A9581159F4108F4D07ED1E0C11116
:1029800001C0D0E01996ED91FC911A97309731F083
:102990001B966D917C9180E00995D823D11539F073
:1029A0008CEF8C0F813A28F58C2F0E94420911156B
:1029B000A9F0E0919104F0919204808584FD0EC00D
:1029C00080919004811551F0808191819C0121506A
:1029D00031092F333E4710F40E945D09D8DA109276
:1029E00092041092910410929004DF91CF911F9164
:1029F0000895CDDA8C2F4ADEDACF962F20916F051D
:102A000022FF0FC0682F660F660F660F692B609359
:102A100028050E94D105AFDA90932A0580932905F5
:102A200008950C94D10590912205292F2823211572
:102A300059F08095892380932205811531F09BDA26
:102A400080932B0590932C05089580E090E0F8CFBB
:102A5000CF93DF93EC018FDA8C1B9D0BDF91CF912D
:102A60000895A0E0B0E0E7E3F5E10C943533162FCC
:102A7000D72FC42FD22E811599F040931F057BDAF2
:102A800090935A0180935901C77081E001C0880F6B
:102A9000CA95EAF7EDDECDB7DEB7E7E00C94513327
:102AA00090911F05491334C0E0905901F0905A01EC
:102AB00062DA9C012E193F097901812F9D2FA5D83B
:102AC000E816F90628F5D0E2DD0DCD1591F0C770B6
:102AD00011E0812F01C0880FCA95EAF7CFDED83008
:102AE00040F48D2D877001C0110F8A95EAF7812F70
:102AF000BFDE60E070E0802FFDDDD83060F62D2D68
:102B0000277081E001C0880F2A95EAF7B7DEC3CFAE
:102B1000C77081E001C0880FCA95EAF7F7CFACE033
:102B2000B0E0E5E9F5E10C942B337C01DC0114966F
:102B30008C91811509F4FDC161E0C7010E947F0CF1
:102B40008C01F7018581811529F180911B059091F8
:102B50001C050097F9F008171907E1F0FC01FF27A1
:102B6000887F9927892B09F0A6C0A4E0EE0FFF1FEC
:102B7000AA95E1F7E556FB4F858184608583118333
:102B80000083CF01B9DE1092270561E0C7010E94E2
:102B90007F0C8C01D70115968C910034BEE71B0782
:102BA00009F099C0811539F080910404811186C023
:102BB00081E080930404D70115968C918111A2C005
:102BC0000115A7E51A0708F4C7C10115B8E51B07E9
:102BD00010F00C94E91E6801E7E5DE1A68E074E085
:102BE0008C2D0E94F00D892B31F5C601E4E0880F91
:102BF000991FEA95E1F7FC01E556FB4F2281213050
:102C000009F069C12091080430910904232B99F03F
:102C100020910A0430910B04232B69F020910C04BD
:102C200030910D0440910E0450910F04242B352B4C
:102C3000232B09F45AC180911204811509F411C2A1
:102C4000C0902305D090220596D988579C4E90932A
:102C5000140480931304F7018581811509F401C2DE
:102C60008D2D8C298D7981112EC20115F0E51F075C
:102C700008F0C9C1011520E4120708F02AC2063E77
:102C8000110509F4EEC1C80190528115904208F077
:102C900027C2D70116968C91803108F40CC2C80166
:102CA0009927109227058D32910509F0C5C182E060
:102CB0008093270519C2E0E0F0E05ECF8091050423
:102CC000811104C081E08093050475CF1092040443
:102CD0001092050470CF0134EEE71E0709F06BCFA8
:102CE000811509F468CF80910604811106C081E046
:102CF000809306048AE18ADC5ECF109206048AE1A2
:102D0000C5DC59CFC80197578038910508F0F7C046
:102D1000003108F0FDC066E472E080E090E00E94BF
:102D2000D20C8111F5C0812C912C5401011146C0A7
:102D300004E09E012F5F3F4F6901D601E02F1D92F5
:102D4000EA95E9F724013501FFEF4F1A5F0A6F0A90
:102D50007F0AC501B4010E94D20C8983811509F450
:102D6000D7C0813009F0B4C0A50194012E5F3F4F58
:102D70004F4F5F4F2D833E834F835887C301B2016E
:102D80000E94D20C182F8A83811509F4C1C08FEFDD
:102D9000810F833078F56D817E818F8198850E94C7
:102DA000D20C8B83811511F0C601BADC24013501E8
:102DB00033E0430E511C611C711C19C0B7E48B1623
:102DC000B2E09B06A104B10409F4A2C0C501B4019C
:102DD0000E94D20CEFEF8E1A9E0AAE0ABE0A811133
:102DE000EDCF0150A3CF4D805E806F80788453017A
:102DF0004201A3CF8BEF810F8330A0F52401350171
:102E000043E0440E511C611C711C6D817E818F81D9
:102E100098850E94D20C8B83811549F3C301B201BE
:102E20000E94D20C8C83811108C02401350154E02A
:102E3000450E511C611C711CDACF8B819C81813045
:102E4000AFEF9A0710F0982F8827163029F0173027
:102E500031F00E94FA21E9CF0E94B821E6CF0E940A
:102E6000D921E3CF143009F0BECF6D817E818F81EF
:102E700098850E94D20C182F24013501B4E04B0E26
:102E8000511C611C711CC501B4016D5F7F4F8F4FD8
:102E90009F4F0E94D20C111509F43AC08115C1F15F
:102EA0008150990B4FEF489F9001499F300D11249D
:102EB000E12FE150FF0B2E0F3F1F2150310908F485
:102EC00096CF8FE99FE00197F1F700C00000F5CFA2
:102ED000C60126DC8CCF223009F0ADCE20910C0447
:102EE00030910D04232B09F4A6CEFC01E056FB4FD4
:102EF00020812E7F208385569B4FFEDC9CCE03379E
:102F0000FCE71F0749F5809112048115B1F0CFDC71
:102F1000809128058770811561F0D70115968C91F5
:102F2000811539F080916F0582FF03C082E00E9415
:102F30007C062C96E1E10C944733109223050E9405
:102F4000A50619D888579C4E9093140480931304B7
:102F500081E080931204DCCF023A22E51207C1F12E
:102F600058F4C80190528115904218F1013E1105A4
:102F700079F1053E110503C0023B52E5150709F042
:102F80005ACE25EE30E02770332781E090E001C073
:102F9000880F2A95EAF72091150430911204311513
:102FA000F9F0F70135813115B1F0282B2093150484
:102FB000AFCFD70116968C91803108F03CCE812F8F
:102FC00099278F7199278230910511F04297D7CFB9
:102FD00021EE30E0D8CF809582238093150498CFDE
:102FE000322F3823311509F426CE982F909592234D
:102FF000909315040E949D06D70115968C9181151A
:1030000009F486CF18CE003EB2E51B0708F046C093
:10301000003CE2E51E0728F5003AF2E51F07E8F458
:10302000003622E51207E8F4C80192558034910574
:10303000C0F010922705C8018E32910508F061C0DA
:103040008832910508F04EC08E31910508F04CC0D1
:1030500004974A9708F42BCE36C0043B32E5130799
:1030600041F7F7013580311409F455C00E35FCE7FE
:103070001F0709F44CC00F352CE7120751F00D352E
:103080003CE7130709F047C080911901811509F445
:103090003EC01092190180E054DC3ACF09374CE76A
:1030A000140728F407375CE71507D8F6C2CF0B37AB
:1030B0008CE71807D5CF812F8F71843191F286313B
:1030C00011F410922705F3DB809115040E949706F6
:1030D000C8CFD70116968C91803108F0E0CDC1CFD2
:1030E000C801DFCD8A9779F780911504811531F0F9
:1030F0008091270592E08927809327050E94C70FBA
:10310000B0CF8C34910581F38D329240ECCF81E0C9
:1031100080931901FDCE80911901811169C0C80108
:1031200097558115914008F0FEC05801F8EFAF2285
:10313000BB24A114B10409F0EBCEF801FF2754E041
:10314000EE0FFF1F5A95E1F79F0125563B4F69018E
:10315000D70115968C91E056FB4F908180FB90F93A
:103160009083811509F4D6C10E94BB0F90931E0570
:1031700080931D05F60182818F5F828380912705F0
:1031800090912305892B8383809122058483468136
:10319000578166857785C6010E941409D601159668
:1031A0008C9181FF5801B0921C05A0921B05D7019C
:1031B00015969C91911509F427C610921F05980148
:1031C00030572332310508F008C684E090E00E94B1
:1031D0000C3490936F0580936E05F801E150F04731
:1031E000E232F10508F0DDC1E858FB4C0C94AB333A
:1031F000380150EE651A710850902405809123051E
:10320000582A80912205582A88E06816710408F02F
:103210005EC098012770332781E090E001C0880FDD
:103220002A95EAF7311409F44FC0582AD7018D9135
:103230009C910E941F0621E030E0F90102C0EE0FD0
:10324000FF1F8A95E2F7FC87EB872091910430916C
:1032500092043E832D834091990450919A045A8799
:10326000498768E1C62E64E0D62EA12CB12C5110FE
:1032700005C0D60112968C9181111BC0F601838185
:1032800090E02B853C8582239323892B91F08085C8
:10329000982F9770911101C087E038E06316710490
:1032A00008F065C0311409F45EC086958170811103
:1032B00063C09FEFA91AB90AAFE0CA0ED11CB8E0EB
:1032C000AB16B104A1F61CC080955822AFCF3110C7
:1032D00037C08091990490919A040817190781F4D6
:1032E00010929A04109299041092950410929604E8
:1032F00010929704109298041092940410929304E0
:103300008091910490919204009709F408CFE8E02D
:103310006E16710408F0E9C0652D0E94CC08811179
:1033200002C081E00EDBF7018581F801E851FC471E
:10333000E730F10508F03BCFE656FB4C0C94AB337D
:1033400010939A04009399040E9451096093950484
:103350007093960480939704909398041092940429
:103360001092930463CF82FB882780F9A0CF311499
:1033700009F49FCF80FF9DCFD6018D909C900815BA
:10338000190519F4311409F494CFED81FE81EC157F
:10339000FD0509F48ECFD6011D96ED91FC91309775
:1033A00021F08081811509F484CF652DC6010E942A
:1033B000CC08811509F47DCF81E00815190509F0C5
:1033C00080E0482E43208114910441F0411006C052
:1033D000E985FA858E169F0609F06BCF80E0B1DA99
:1033E000D0929204C092910481E0809390048FE087
:1033F0008A9DF0018B9DF00D1124E85EFB4F8581C5
:103400008093170441100EC08114910459F08081FB
:1034100091819C0124503109213A310508F049C0BD
:103420000E9442098FE08A9DF0018B9DF00D1124CE
:10343000E85EFB4FC680D780C6019A9581159F41F3
:1034400010F420EED22299249394C60101978F3371
:103450009E4708F0912C8FE08A9DD0018B9DB00D86
:103460001124A85EBB4F1996ED91FC911A973097E5
:1034700031F01B966D917C9181E009959822911411
:10348000A9F08FE08A9DF0018B9DF00D1124E85E7C
:10349000FB4F868197810E947E0580931604C601AA
:1034A00048E06416710438F40E945D090E94C70F59
:1034B0000BC0ECD8B7CF0497813A910558F46C2D26
:1034C0008EE491E00E942809411409F428CE0E945C
:1034D000C70F1ECD0E94C70F8FE39CE90197F1F73C
:1034E00000C000008C2D92D8EFCFDC012D913C91D3
:1034F0000217130739F4311008C01092900480E0CD
:1035000020DA0DCE311409F40ACEFC01808585FD48
:1035100006CEF5CFF9014485558566857785C901C5
:103520000E941409D60115968C9181FF40CEC601E8
:10353000C7D980911B0590911C050817190709F040
:1035400036CE10921C0510921B0531CE06E221EEFC
:1035500041EE6AE17CE785DADBCC07E225EE45EE59
:103560006BE17CE7F8CF06E221EE40EE68E17CE714
:10357000F2CF07E225EE44EE69E17CE7ECCF06E20C
:1035800021EE42EE6CE17CE7E6CF07E225EE46EE67
:103590006DE17CE7E0CF08E221E045EE6EE17CE7FB
:1035A000DACF80916E05816080936E0560916E0523
:1035B00070916F0584E090E00E943A340E941D10E3
:1035C000A7CC80916F05886080936F05EFCF8091C5
:1035D0006E058260E9CF80916E058460E5CF8091B1
:1035E0006E058860E1CF80916F058160EDCF80919D
:1035F0006F058260E9CF80916E058061D5CF8091A3
:103600006E058062D1CF80916E058064CDCF0E941F
:103610001D1080916E058068C7CF80916E058C600B
:10362000C3CF80916F058360CFCF80916E058E7F71
:10363000BBCF80916F05877FC7CF80916E058D7F4F
:10364000B3CF80916E058B7FAFCF80916E05877F62
:10365000ABCF80916F058E7FB7CF80916F058D7F47
:10366000B3CF80916E058F7E9FCF80916E058F7D49
:103670009BCF80916E058F7B97CF0E941D1080910C
:103680006E058F7791CF80916E05837F8DCF80916E
:103690006F058C7F99CF80916E05992782FF939556
:1036A00090FB82F990FB83F97FCF80916F05982F73
:1036B000909590FB80F990FB81F986CF90916E05F3
:1036C000892F8F7B96FF80646FCF0E941D10909191
:1036D0006E05892F97FB87F9805866CF61E08EE0F1
:1036E00090E00E94203462CF60E0F9CF90916E05A7
:1036F000892F8F7E94FF806157CF90916E05892F1F
:103700008E7F90FF816050CF90916F05892F877FCA
:1037100093FF886059CF89E282C3980134572034DF
:10372000310508F4F5CB0737BCE71B07F9F008377C
:10373000ECE71E0731F19801205E32452032310559
:1037400028F5911123C00F7181E090E09C0102C027
:10375000220F331F0A95E2F78901622F83E090E080
:103760000E942034802F0E94C405D2CB81E09115A5
:1037700051F00E94D10543E062E081E00E945306CF
:10378000C7CB82E0F4CF0E94DB05F5CF4091210545
:1037900080912605282F30E02095309570E0242375
:1037A0003723232B19F04823409321050B373CE79F
:1037B000130741F4911509F4ABCB0E94B1050E94A7
:1037C000ED08A6CB003442E5140708F056C00032DD
:1037D00052E5150708F058C0011580E5180758F59F
:1037E0000115A0E41A0708F065C0911509F47AC024
:1037F0000A35FCE71F0709F4FFC008F0E3C00130F9
:103800003CE7130709F4F6C003304CE7140709F44A
:10381000EBC001155CE7150709F064C00E941D109C
:10382000AFEFB4E3ECE0A150B040E040E1F700C0FE
:1038300000000E949E099801305521153240A8F6DB
:10384000980145E0369527954A95E1F7822F8F70CC
:103850002091210530E041E050E0082E02C0440FE5
:10386000551F0A94E2F724233523232B09F4BDCFF7
:103870009111A5CF109223052ACE9801205C3245E4
:103880002032310508F0B1CF802F8F7120912105B2
:1038900030E041E050E0082E02C0440F551F0A946A
:1038A000E2F724233523232B09F49FCF911509F444
:1038B0002FCB85CFF7018681803108F096CF91110B
:1038C00011C0212F2F7081E090E002C0880F991F56
:1038D0002A95E2F72091210530E082239323892B5A
:1038E00009F016CBF7018581C080D180811509F4DC
:1038F00087C0C6010E94560C182F682FC6010E946F
:10390000E905B601812F0E943B0C0E94A307D82E27
:10391000192FD7011596AC9015971696BC90B294B6
:103920008FE0B822809128058770811509F1CA2C93
:10393000A114F9F0892F807F803469F080E28D0D29
:103940008830B0F0892F807E803229F4B2E0DB1617
:1039500078F0B11469F080916F0582FF09C082E0B0
:103960000E947C06809128058770CC24C394811125
:10397000C12C812F82958F70883009F428C108F0FE
:1039800044C0823008F453C0825F8F70823008F4E4
:1039900084C0C11409F44AC18091280580FD46C144
:1039A000D70115961C928695869586950E94D1051D
:1039B000C701B5D8809128058695869586950E9481
:1039C000DB0534C10B358CE71807C1F080916F051A
:1039D000002482FF0394802D0C359CE7190709F021
:1039E00081CF0E94CF0B7ECF6FEF7FEF80E090E022
:1039F0000E943A340E94291081E0F3CF80E0F1CF99
:103A0000C6010E941F06182F7CCF893009F452C1CD
:103A10008A5F8F70823008F0BCCFE2EFDE125BC1AC
:103A2000812F8F71A11054C10E94D105FDC0012FBB
:103A30000F70103110F00295007FA114A9F001154C
:103A400059F080E28D0D883010F0D11007C0802F22
:103A50000E9497060E94C70F8D2D40C080912705B8
:103A6000802B80932705F6CF8D2D0E9446130115DC
:103A700009F48FCF80E28D0D883010F0D11004C092
:103A8000802F0E949D0606C0009580912705802307
:103A9000809327050E94C70F7CCF012F0F70107FE6
:103AA000103211F00295007FD11451F0F1E0DF16D1
:103AB00009F46CC0A11409F478C0B114E9F0CCCFBA
:103AC00080916F0582FD14C0A11459F0011529F0F1
:103AD000802F0E9497060E94C70F80E00E94061365
:103AE00058CF80E00E944613011509F452CFC8CF89
:103AF000A11471F1B11004C0802F0E94381449CF75
:103B000021E0B21211C010912205802F81230817E5
:103B100009F43FCF0E94BB0F90932C0580932B0597
:103B2000102B1093220535CF35E0B31232CF802F02
:103B30000E943814802F0E94131580912405902F25
:103B40009823091709F425CF802B8093240521CFD2
:103B5000B11012C0802F0E943E14802F0E941315B6
:103B600080912405902F9823911509F412CF009588
:103B70000823009324050DCF41E0B4120ACF8091B1
:103B800023058023811509F404CFE4CFA11429F083
:103B900056E0B51608F0FDCEAFCF85E0B81608F0B8
:103BA000F8CE802F0E943E14F4CEB114D1F399E3E5
:103BB000D91209C0AFEFB7EEE3E0A150B040E0404A
:103BC000E1F700C000008D2D0E944613E2CE812F48
:103BD0008370811138C0A11027C04D2D42954695A4
:103BE0004770440F440F8D2D8F70042E01C0880F35
:103BF0000A94EAF72D2D2071D4FE07C02FE030E0A3
:103C000001C0220F4A95EAF7209516951695137074
:103C10001230A1F0133081F030912505113059F0A8
:103C2000822B83230E94C4050E94190960E0C7010A
:103C30000E947F0C7EC9832B822BF4CF822B909124
:103C400025058927EFCFA11451F110FFEDCF4D2DA0
:103C5000429546954770440F440F8D2D8F70042E6A
:103C600001C0880F0A94EAF72D2D2071D4FE07C0F9
:103C70002FE030E001C0220F4A95EAF72095169513
:103C800016951370123089F0133069F030912605C3
:103C9000113041F0822B83230E94C705C5CF8230AB
:103CA00018F2D5CF832B822BF7CF822B909126054C
:103CB0008927F2CF1F70A11439F0812F0E94D105FE
:103CC0008D2D0E943814B0CF8D2D0E943E14812F6F
:103CD0000E94DB05A9CFF3EFDF1680F420EFD216A8
:103CE000E1F031EFD316A1F0A11409F460C0B114D2
:103CF00009F45AC08D2D0E94061396CF43EFD416B7
:103D0000F1F054EFD512F0CF80916F0582FD23C002
:103D1000812F8F71A114E1F287CEA11469F085E0A3
:103D2000B81608F081CF1F7181E090E0012E01C02C
:103D3000880F0A94EAF7BACF96E0B916F2CF80E07E
:103D4000A11409F4A9CF1F7181E0012E01C0880FD1
:103D50000A94EAF7A1CFA114C1F0809128058770D9
:103D6000843049F41092280510922A0510922905F2
:103D7000812F8F71ADCFA5E063E0BA1608F054CF64
:103D8000812F8F710E94FD144FCFB5E0BB1640F01C
:103D90001092280510922A051092290564E0F0CFB0
:103DA00081E00E947C0640CF812F8F713DCEB114FF
:103DB000F9F2E9E3DE1209C0FFEF27EE33E0F1503C
:103DC00020403040E1F700C000008D2D0E944613D6
:103DD0002BCF0337BCE71B0713C90631ECE71E07DF
:103DE00009F09BCC809123058A7A91E0811101C072
:103DF00090E09093200565E3811101C069E28EE4B3
:103E000091E00E94280963CB0631FCE71F0709F007
:103E100084CC80912005811509F47DCC85E30E9436
:103E2000420955CBA0E0B0E0E8E1FFE10C94353366
:103E300080916D05803108F049C080916C05811535
:103E400009F444C0C0912E0587E0D82E80912D053D
:103E50008C17E1F1EC2EF12CDC9EE0011124FE0127
:103E6000E15DFA4F84818115B1F1918180916805FE
:103E7000981331C090818091670598132CC085817B
:103E8000811129C0028113818091690590916A0591
:103E9000081B190B60E087E695E00E947F0C0E94EA
:103EA000050E08171907B8F480916D058F708061B1
:103EB00080936D05CB5CDA4F88818F708061888339
:103EC00087E695E00E948F150E947206CDB7DEB797
:103ED000E7E00C945133E7012196C770B7CFADE00E
:103EE000B0E0E5E7FFE10C942D338C0186E0F801AA
:103EF000DE01189601900D928A95E1F7F801F580A0
:103F0000E48087E6882E85E0982E80916B058111EC
:103F100017C0E11491F0F11409F455C1C8010E94D1
:103F2000A70C811509F44FC187E0F801A7E6B5E0B9
:103F300001900D928A95E1F775DFFF24F39461C03B
:103F4000A280B380D0906C058091690590916A053C
:103F50003501681A790AD11409F4F0C0C080518083
:103F600060E087E695E00E947F0C0E94050E6816CF
:103F7000790608F09EC0E11401F380916805F8010C
:103F80009181E0906D05F0E1EF1608F05BC09813A9
:103F900017C090916705F8018081981311C0F11046
:103FA0004BC08E2D8F70806180936D0587E695E004
:103FB0000E948F1580916D05F8018683F12C21C038
:103FC000F1103AC040E0652D8C2D0E94580B40E066
:103FD000652D8C2D0E94580BF82E8111EFCF88850E
:103FE00099850E949B0C292F22952F70903470F494
:103FF0009F702230A0F09115B1F0F80196819031B8
:1040000090F48F2D2D96EFE00C9449332A5F2F709A
:10401000223068F0C8010E948F15FD2CF2CF911557
:1040200011F0811571F3805E883058F3F3CF803F33
:1040300040F3815F8330F9CF80916D05816080937B
:104040006D05BCCF981315C090916705F80180816C
:1040500098130FC0F1100DC0E682C8010E948F15A1
:1040600087E0F801A7E6B5E001900D928A95E1F7A7
:1040700064CFC8010E94A70C811509F4A4C0F114F3
:1040800009F4A1C080916D05803208F44DCF809174
:104090006705909168059A838983BC82AB82809181
:1040A0006B058D831E82EF82CE0101960E948F15D3
:1040B0003BCFD0906D05F0E1DF1650F487E695E038
:1040C0000E948F1587E0F40111928A95E9F776CF67
:1040D000E11409F432CF90916805F80181819813B9
:1040E00011C090916705808198130CC0F1100AC02F
:1040F000D682C8010E948F1587E0F40111928A953B
:10410000E9F71BCFC8010E94A70C811509F45BC019
:10411000F11409F458C080916D05803208F404CF81
:1041200080916705909168059A838983BC82AB82F0
:1041300080916B058D831E82DF82B6CF60E087E6BB
:1041400095E00E947F0C0E94050E6816790608F023
:10415000B9CFE11409F4F1CEF114A9F190916805F9
:10416000F8018181981325C090916705808198138B
:1041700020C08091690590916A05A81AB90AF8ECE7
:10418000AF16B10408F06CCF80916D0580FD68CF4B
:10419000803108F465CFF8018683982F907F903F97
:1041A00009F45BCF982F907F905F8F70892B868367
:1041B00054CFC8010E94A70C8111B6CE80916D0525
:1041C000816080936D05C8010E948F15B6CEABE16A
:1041D000B0E0EDEEF0E20C9438334E8B5F8B688FDD
:1041E000798F8A8F192F9B8F9111109227051D8A25
:1041F00086E0FE017696DE011F9601900D928A956B
:10420000E1F70A8D80916F0582FF1FC00E94BB0FEE
:104210002091290530912A05821B930B8838934100
:1042200038F08091280582FD03C082E00E947C0660
:104230000E94BB0F20912B0530912C05821B930B04
:104240008838934110F00E94A506011561F00B8B90
:104250001C8B61E0CE010F960E947F0C61E0CE01C5
:104260000F960E947F0C0B8B1C8B87E0FE013F9604
:10427000DE01189601900D928A95E1F7CE0108961D
:104280002EDE811110C020912D0530912E0587E082
:10429000FE013896DE01119601900D928A95E1F7A4
:1042A0008C8581110BC017E080912E0590912D0512
:1042B00089132BC06B96E4E00C945433822F90E06A
:1042C0000196877099273817190671F40E941D10FE
:1042D00010922D0510922E0587E0E7E6F5E0DF014C
:1042E0001D928A95E9F7DFCF97E0929FD0011124C4
:1042F000A15DBA4FFE01319601900D929A95E1F7BA
:1043000080932D050E947206CECF189FC001112404
:10431000815D9A4FE4DD811569F280912E0590E070
:1043200001968770992780932E05BECFA6E0B0E056
:10433000ECE9F1E20C9438330E94BB0F8C018091C0
:10434000EC039091ED038017910771F019821A82A6
:104350000E94BB0FBC0149815A8180E090E037DFA9
:104360001093ED030093EC032696E4E00C94543391
:10437000A6E0B0E0EEEBF1E20C943A339093E9035F
:104380008093E803811520E2920730F40E943113F4
:104390002696E2E00C94563380EF89838A830E944C
:1043A000BB0F8160BC0149815A8181E091E00FDF40
:1043B000EFCFA6E0B0E0EFEDF1E20C943A3390934A
:1043C000E9038093E803811520E2920730F40E940C
:1043D0005E132696E2E00C94563380EF89838A833D
:1043E0000E94BB0F8160BC0149815A8181E090E04D
:1043F000EEDEEFCFCF93DF93D82FC92FB9DF8D2F0C
:104400009C2FD7DFDF91CF9108950F931F93CF9308
:10441000DF938C01862F68E074E00E94F00D892BF9
:1044200091F4C0910804D0910904209761F0F8013B
:104430008281833039F4CE01DDDFCE01DBDFCE01B6
:10444000D9DF01C0E0F7DF91CF911F910F9108955F
:104450000F931F93CF93DF938C01EB0168E074E01F
:104460008C2F0E94F00D892B09F057C0FE01FF2709
:10447000D80112968C911297E058FE4F8130A9F422
:1044800015968C9182FD4EC080FF4CC082E08083E7
:1044900080910A0490910B040097B9F4809108046C
:1044A000909109040097C9F110C08230A1F51596CA
:1044B0008C9182FD26C080FD0AC083E080838091BC
:1044C0000C0490910D040097F1F052DF26C084E0B7
:1044D000808380910E0490910F040097B1F7809132
:1044E000080490910904009701F184DF80910A0487
:1044F00090910B04009749F780910804909109046A
:10450000E4CF85E0808380910804909109040097AE
:1045100021F070DFF1CF86E08083DF91CF911F9192
:104520000F91089581E08083B9CF80910A04909122
:104530000B04B8CF0F931F93CF93DF938C01EB0144
:1045400068E074E08C2F0E94F00D892B71F4DD2758
:10455000C058DE4F8881F801128218828330E9F05A
:1045600048F4813059F0823081F0DF91CF911F9172
:104570000F9108958430B1F08530B9F78091080427
:1045800090910904009789F306C080910A049091E4
:104590000B04009799F30DDFE8CF80910C04909104
:1045A0000D04F7CF80910E0490910F04009799F7B6
:1045B000209108043091090480910A0490910B0421
:1045C00021153105F9F2009731F7C901E4CFA6E0D2
:1045D000B0E0EDEEF2E20C942D33FE01319686E070
:1045E000DF011D928A95E9F788E3E82E81E0F82E35
:1045F0008F019EE3C92E91E0D92E3F01AA24A394F6
:10460000B12C33E4832E31E0932EF70181917F01A9
:104610008F3F09F43EC0F894E82FE295EF70F0E088
:1046200021A18F70A50102C0440F551F8A95E2F7A2
:10463000CA01922F982B91A392A18095892382A3DE
:10464000789400C0EEE3F1E031E0512C21912F3F4E
:1046500079F0A22FA295AF70A05EB0E08C9190E0AF
:104660002F7002C0959587952A95E2F780FF35C097
:1046700080E0582A330F8E169F0641F7F70182918A
:104680008F3F11F00E948E0850EA5A95F1F7D80139
:104690005C920F5F1F4FCE14DF0409F0B6CF46E0E7
:1046A00050E0B30188E891E00E94E033892BB9F033
:1046B00086E0F301A8E8B1E001900D928A95E1F758
:1046C00081E0809358010E94BB0F90935701809323
:1046D00056012696EFE00C944933832FCACF809180
:1046E00058018115B1F300915601109157010E94B4
:1046F000BB0F801B910B059760F346E050E068E824
:1047000071E081ED93E00E94E033892B49F086E06F
:10471000E8E8F1E0A1EDB3E001900D928A95E1F7B0
:1047200010925801D6CFCDB7DEB7AE970FB6F8943A
:10473000DEBF0FBECDBF85B7806885BF85B78068F7
:1047400085BF84B7877F84BF0FB6F894A895809102
:104750006000886180936000109260000FBE80E866
:1047600090E00FB6F89480936100909361000FBEC3
:1047700081E0809305018CE898E090934D0180934F
:104780004C010E94B4080E94710D0E945B0A0E94B5
:10479000FE0A8091E20084608093E2007894809128
:1047A000D903811599F08091E9001091EC008F7088
:1047B000179511271795182B1092E9008091E800A2
:1047C00083FD0E943E101F701093E90082E084BDBB
:1047D00093E095BD9AEF97BD80936E000E94E30C25
:1047E000811102C00E949B0E08E311E09EE3E92EB6
:1047F00091E0F92ED8018D918D018F3F11F00E942B
:104800008E08E016F106B1F70EE311E083E4E82E1E
:1048100081E0F82EF80181918F018F3F11F00E9405
:104820008E08E016F106B1F786E0E1EDF3E0DF0176
:10483000282F1D922A95E9F7E8E8F1E0DF011D92A3
:104840008A95E9F780E090E00E940C34833E9E4F09
:1048500021F40E94E30C811129C063EE7EEF80E019
:1048600090E00E943A3460E082E090E00E942034C0
:1048700081E08093250561E083E090E00E94203490
:1048800060E074E184E090E00E943A340E949B0E64
:1048900040E050E0BA018FE090E00E94323440E006
:1048A00050E0BA0183E190E00E94323482E090E06F
:1048B0000E9404348093900184E090E00E940C34C4
:1048C00090936F0580936E0582DEEFEFF6E721E0AF
:1048D000E150F0402040E1F700C0000078DE809118
:1048E000D10380FF08C06FEF7FEF80E090E00E946F
:1048F0003A340E949E0983E090E00E9404340E94B2
:10490000C405809126050E94B105809307040E948A
:104910005A051092C20380E88093A1010E942E2FB5
:104920006BE070E08CED98E00E94200E811509F498
:104930003FC08091C20365E070E081FDA9C087EDB2
:1049400098E00E94200E811599F16DE070E085ECF1
:1049500098E00E94200E811559F10E945109DC0156
:10496000CB01805A9541AF4FBF4F8093C6039093C0
:10497000C703A093C803B093C903E2ECF1E080E061
:1049800092E0DF019C011D9221503040E1F7F0934D
:10499000A001E0939F018FEF9FEF9093C503809359
:1049A000C40381E08093CB038093CA031092C303B6
:1049B00084988C9885988D988091900183608093DD
:1049C0009001529A539A5A9A5B9A0E946A0581E022
:1049D00080930404109205041092060410920704B8
:1049E00086E091E09093EF038093EE0333243394B9
:1049F000222423948091D90310E4853009F47FC0E8
:104A0000E6DD01E911E0B1EDEB2EB3E0FB2ED701BD
:104A1000F80191918D9127E931E02E173F0709F4B4
:104A200078C09817B1F3D12CD701CD907D01F80152
:104A300091908F019C1419F19C24B12CAA24A39469
:104A4000892D8A218115A1F0B982DA820E94BB0FDB
:104A50009C838B832D8291E08C2D8A21811101C052
:104A600090E09E8349815A816B817C818D81AFDB8F
:104A7000B394AA0CF5E0BF12E3CFF801C292D3942D
:104A800026E0D212D1CF0E945109DD24D39445C033
:104A900082ED98E056CF8091D903843029F10E94AD
:104AA0002D0E10928E0188E190E00FB6F894A89533
:104AB000809360000FBE1093600083B7817F846095
:104AC00083BF83B7816083BF7894889583B78E7FD7
:104AD00083BF0FB6F894A895809160008861809399
:104AE0006000109260000FBE72DDE1EDF3E0819195
:104AF000811193C7A7EDB3E0AE17BF07C1F780914F
:104B0000D903853009F4C7CF0E941D100E941909EE
:104B100077CF981388CF0ADCD12C009193041091A1
:104B200094040115110591F180909B0190909C01D6
:104B3000A0909D01B0909E010E94510968197909C9
:104B40008A099B098090970190909801A090990103
:104B5000B0909A01681579058A059B05B8F0C801DF
:104B60000E943113109294041092930410929B01AE
:104B700010929C0110929D0110929E01109297013B
:104B8000109298011092990110929A01E0901B05E1
:104B9000F0901C05E114F10439F1A0901D05B090CE
:104BA0001E050E94BB0F8C010A191B09C7010E9438
:104BB000050E80179107C0F420911B0530911C054C
:104BC000C9019927287F3327232B09F00AC2A4E0C3
:104BD000880F991FAA95E1F785569B4FDC01159622
:104BE0002C9122FF0E947C1480911204811569F09F
:104BF0000E94BB0F2091130430911404821B930B6D
:104C00008F3F9F4710F40E9457148091CB0381156A
:104C100009F4A3C082EC91E09093A00180939F01DE
:104C20001091070400910404F090050484E499E0D5
:104C30000E946D0F87E399E0123051F08EE299E007
:104C4000133031F08CE399E0113011F086E299E0F5
:104C50000E947A0F8BE199E00E946D0F8EE099E03F
:104C6000F11006C089E099E0011102C080E099E0EE
:104C70000E947A0F133009F0BCC1E090DE03F0907F
:104C8000DF030091E0031091E1038BEF98E00E94B5
:104C90006D0FC7010E94880A0E947D0F84EF98E083
:104CA0000E946D0FC8010E94880A0E947D0F81E05A
:104CB0000E943F0F89EE98E00E946D0F20917605CB
:104CC0009091770580917805C090790530917505B0
:104CD00039832A839B838C838E010F5F1F4FFBE1F7
:104CE000EF2EF1E0FF2E5E01E5E0AE0EB11CD80123
:104CF0008D918D01811509F477C1F7018081C11073
:104D00008F7D0E94C00EFFEFEF1AFF0AA016B106BA
:104D100071F782E299E00E947A0F8091C40390912A
:104D2000C503892B09F06AC18091CA038115A9F0D6
:104D30000E9451090091C6031091C7032091C80336
:104D40003091C903601B710B820B930B6F3F7F4F38
:104D50008F4F9F4710F40E942D0ED1100E943E0EDF
:104D600084EF0E94D82E092E000CAA0BBB0B925088
:104D7000A109B1096C017D01A1E0BEEFA701960177
:104D80000E94C43361303EEF73073FEF8307930700
:104D90000CF417C220E032E040E050E00E948F3374
:104DA00050954095309521953F4F4F4F5F4F2130A3
:104DB0008EEF38078FEF480758070CF0F4C141E039
:104DC0005EEF6FEF7FEF8091E3039091E403841730
:104DD000950731F05093E4034093E3033092E703E7
:104DE00085EFE6D7092E000CAA0BBB0B9250A10948
:104DF000B1096C017D01A1E0BEEFA70196010E94FF
:104E0000C4336130FEEF7F07FFEF8F079F070CF47D
:104E1000FAC120E032E040E050E00E948F3350952C
:104E20004095309521953F4F4F4F5F4F2130AEEF6A
:104E30003A07AFEF4A075A070CF0D7C141E05EEFDF
:104E40006FEF7FEF8091E5039091E603841795075C
:104E500009F0C4C18091E7038115E1F08091EE0370
:104E60009091EF03892BA1F08091E3039091E403EB
:104E70009A8389838091E5039091E6039C838B83D9
:104E800044E050E0BE016F5F7F4F84E00E94770BEB
:104E90001092E7030E9419099091CC03891721F021
:104EA0008093CC030E9451098091D903843009F486
:104EB000B5C110910404111509F49CCD509005045E
:104EC0006091E3037091E403072E000C880B990BAB
:104ED0000E94DB32762E872E982EA92E6091E50354
:104EE0007091E603072E000C880B990B0E94DB32B1
:104EF000B62EC72ED82E092F272D382D492D5A2DE5
:104F0000672D782D892D9A2D0E94AB32462E672E63
:104F10007C012B2D3C2D4D2D502F6B2D7C2D8D2D5F
:104F2000902F0E94AB329B01AC01642D762DC701FE
:104F30000E9430320E94EE310E94AD327B017093AC
:104F4000DD036093DC03272D382D492D5A2D6B2D61
:104F50007C2D8D2D902F0E94533020EE3EE245E6B1
:104F600052E40E94AB3220E030E044E353E40E947C
:104F700030320E94AD32CB018C599F4F68E671E010
:104F80000E9416339093DB038093DA034091DA0397
:104F90005091DB036091DC037091DD034093DE03ED
:104FA0005093DF036093E0037093E10324E6E2167D
:104FB000F10408F423C5009709F4B2C48B359105B8
:104FC00008F4B7C410927505863B910508F0B9C482
:104FD00021E0209376058838910508F008C510E097
:104FE000A4C480E090E0FACD87EE98E00E946D0FB7
:104FF0008ACE84E299E00E947A0F8BCE8091CB0317
:10500000811509F491CE8091C30381118DCE0E9448
:105010003E0E2091C4033091C5032115310509F4DA
:1050200083CE10E041E050E0812F90E07A01012E24
:1050300002C0EE0CFF1C0A94E2F7B701622373234F
:10504000672B11F41F5FF0CF2091C20320FF98C09F
:10505000912F990F990F990F37E0390F80E023E0D6
:105060009093140180931701309315012093180138
:1050700024E630E047E050E062E171E088E724D7C1
:10508000892B09F051CE20E2129FA00111248091BA
:10509000C20380FF81C0E2EAF1E080E2DF011D92FD
:1050A0008A95E9F7E7E4F1E0FCA7EBA703E411E058
:1050B0007BE4872E71E0972EABA5BCA56D91BCA7B4
:1050C000ABA7F80181918F01840F952F911D9C0151
:1050D0002E533E4F2901E62FF0E0EE55FE4F20E023
:1050E00030E067E0662E621ACC24C394022E01C021
:1050F000CC0C0A94EAF7520190E0D5018D915D0144
:105100008C21662D691B677070E0B82F062E01C0D8
:10511000BB0F0A94EAF7719561957109677077275B
:1051200001C086956A95EAF78B2B6081862B808378
:105130009F5F983011F72F5F3F4F31962830310530
:1051400081F6EBA5FCA58E169F0609F0B5CF04E607
:1051500010E020E230E042EA51E060E488E748D71E
:10516000892B09F0E1CDE094F0948091C4039091F3
:10517000C5038E219F219093C5038093C403D4CD92
:105180009695879596958795282F912F9295990FAB
:1051900090763FE1390F64CF4E535E4F04E610E046
:1051A00020E230E0DACFBA01A901411592E05907B7
:1051B000610571050CF407CE4FEF51E060E070E03F
:1051C00002CEAFEFB1E0A70196010E94B8332FEFF6
:1051D00031E040E050E00E948F33E9CD5093E60388
:1051E0004093E5033092E70339CEBA01A901411596
:1051F000B2E05B07610571050CF424CE4FEF51E07E
:1052000060E070E01FCEAFEFB1E00E94B8332FEF47
:1052100031E040E050E00E948F3308CE83E080937D
:10522000E9008091E80082FF44CE8091E80090E0A0
:1052300085FF05C00E942A0A811521F191E0809125
:10524000E8008B778093E800911509F432CE009145
:10525000EA031091EB03E9810115110579F1EE3FA5
:1052600009F050C08A81833020F08550833008F0E7
:1052700049C0EA81EE3008F045C0F0E0EF55FB4C44
:105280000C94AB3300E210E0FE0131967F01809177
:10529000E80085FD0AC08091E8008B778093E800E4
:1052A0000E942A0A811599F3C9CF8091F100D70194
:1052B0008D937D010150104051F7C0CFE43150F47F
:1052C000E11551F0E150E33138F4F0E0E155FB4CE9
:1052D0000C94AB33EE3F69F28FEF898313C01A82CF
:1052E00089E08B830FC08A81823089F08330C1F0DE
:1052F000813091F70E9451090E94B1336B837C8306
:105300008D839E83CE0101960E947A0AD2CD88E2D7
:1053100090E00E9404341B821C821D828E83F2CF97
:105320008091D7039091D803892B61F386E0E1ED5A
:10533000F3E0DE01139601900D928A95E1F7E2CF3A
:105340008A81823049F66B817C818D819E810E94A9
:10535000B13388E290E00E942034D4CF4C816B813D
:105360008A810E940C0C9827892798279E838D8319
:10537000C9CF2D813E813227232732274C816B8173
:105380008A810E94E50BBECF0E94FC0CBBCF80E15E
:105390008A83B8CF82E08A8387E4A3CF8C818D3162
:1053A00008F0B0CF8A809B80982489249824A12C6F
:1053B000B12C8E010F5F1F4F7801E80EF11C0E1506
:1053C0001F0509F49FCF80E0B7E48B16B2E09B067F
:1053D000A104B10428F4C40187549E4F0E940434F0
:1053E000F80184830F5F1F4FFFEF8F1A9F0AAF0AE8
:1053F000BF0AE5CF8091D7039091D803892B09F498
:1054000081CF8C818D3108F07DCF882E912CA12CFD
:10541000B12CCA80DB80DC24CD24DC24E12CF12CEF
:105420008E010F5F1F4F412C512C3201481459043B
:105430006A047B0408F066CF27E4C21622E0D20695
:10544000E104F10440F4D80114966C91C60187542C
:105450009E4F0E942034BFEF4B1A5B0A6B0A7B0AF7
:10546000EFEFCE1ADE0AEE0AFE0A0F5F1F4FDECF05
:105470000E94600E47CF84E08BCF8C818D3108F085
:1054800041CF882E912CA12CB12CCA80DB80DC244A
:10549000CD24DC24E12CF12C412C512C32018E0145
:1054A0000B5F1F4F481459046A047B0408F02ACF8D
:1054B00080E0F0EFCF16D104E104F10420F4C6013E
:1054C00089960E940434D8018D938D01BFEF4B1A49
:1054D0005B0A6B0A7B0AEFEFCE1ADE0AEE0AFE0ABF
:1054E000E1CF2C81022F10E02D3108F00BCF8A8103
:1054F0009B819827892798272C01612C712C803F4C
:10550000910508F0FFCE822E912CA12CB12C40EFFA
:1055100050E060E070E044195509660977094217C8
:1055200051056105710508F4EDCE2091D703309146
:10553000D803232B09F042C09C01275D3F4F3EA7B3
:105540002DA780FBEE24FF24E0F880FF0CC0889696
:105550000E9404349D8189279827892781159C47BB
:1055600011F48FEF8D83D501C401840D951DA61D07
:10557000B71D80FF1BC0680181E0C81AD108DE0199
:105580001596AC0DBD1DBCA7ABA78DA59EA5800F24
:10559000911F0E940434EBA5FCA5908181159C47C6
:1055A00021F48FEFABA5BCA58C938601FE0131964B
:1055B000EE0DFF1D2FEFE016F10638F08E010F5FA4
:1055C0001F4FC12CD12C760125C094818581811576
:1055D0009C4711F42483258332E0E30EF11C3296BC
:1055E000EACF80EF481651046104710438F4D80101
:1055F00014966C91C20189960E942034BFEFCB1A99
:10560000DB0AEB0AFB0AEFEF4E1A5E0A6E0A7E0A0D
:105610000F5F1F4FC814D904EA04FB0410F372CEC5
:105620008091D7039091D803892B09F46BCECE01DA
:1056300001960E947A0AFFEF21EE34E0F1502040FB
:105640003040E1F700C0000054C988E0E0E2F1E03A
:10565000DE01919601900D928A95E1F7FE01329656
:105660008FE1DF011D928A95E9F786E0898388E062
:105670007F96DE0115965FCE8CE2898381E08A8376
:105680001B821C823FCE8B819C81092E000CAA0BB1
:10569000BB0B25E0880F991FAA1FBB1F2A95D1F7C6
:1056A000AC01BD01405E5F4F6F4F7F4F48175907F8
:1056B0006A077B0708F426CE8C32E1E09E07A1053D
:1056C000B10508F01FCE4D32F1E05F0761057105AD
:1056D00020F04CE251E060E070E0481B590BBC0147
:1056E000645B764FCE0101960E94D7330BCE4AE120
:1056F00050E06FEF70E0CE0107960E94ED3380918D
:10570000D70389830A8384E08B831C828D8383E0A3
:1057100005CE81E090E09093EB038093EA0382E36F
:1057200090E09093D0038093CF030E94BB0F90939F
:10573000CE038093CD03E6CD0115110571F1D09014
:10574000D503E090CD03F090CE030E94BB0F8E19DD
:105750009F098536910540F1D3FE26C0D0FE24C0B6
:105760000E94BB0F9093CE038093CD038091CF0313
:105770009091D00301979093D0038093CF03892B0E
:1057800061F41092EB031092EA0381E090E09093B1
:10579000D8038093D70300E010E08091D70389837A
:1057A0000A838091CF039DCD82E390E09093D00354
:1057B0008093CF03F2CF1092D8031092D703A2CDDB
:1057C00040E250E06FEF70E0CE0101960E94ED33B1
:1057D00099CD8B81823009F451C078F4811137C0A2
:1057E000FE0132968EE1DF011D928A95E9F788E08D
:1057F00089838B8383E088A385CD853009F473C0CA
:10580000863009F07FCD1C818AE0FE013596DE01ED
:10581000919601900D928A95E1F78BA19CA10E942F
:10582000A7089CA38BA38FEF183068F4FAE01F9FA2
:10583000B001112467597E4F4AE050E0CE018196B5
:105840000E943E3480E089830E94710D5BCD8C8183
:105850009AE0F92E8E010F5D1F4FF8012F2D119246
:105860002A95E9F7B8010E94F00D8983F801DE015D
:10587000129601900D92FA94E1F744CD1C818AE0D2
:10588000FE013596DE01919601900D928A95E1F721
:1058900089A19AA10E94A7089AA389A38BA19CA180
:1058A0000E94A7089CA38BA38DA19EA10E94A7087C
:1058B0009EA38DA38FA198A50E94A70898A78FA348
:1058C0008FEF183060F43AE0139FB0011124675E47
:1058D0007E4F4AE050E0CE018196D0D780E08983A8
:1058E0000E94B4080FCD2C816AE0CE018196DC01C4
:1058F000E62F1D92EA95E9F7283080F4629FB00107
:10590000112467597E4F4AE050E06ED780E08983CA
:105910008AE0FE01B196DE0112960DCD8FEFF7CF32
:105920001092750510E010927605312F10E020E0FE
:1059300012C0309275058E329105A8F3309276052B
:10594000F4CF109276058F3031E0930708F44FC002
:1059500010E030E021E01093770521702093780566
:10596000311107C021E08C33914008F420E02093EE
:10597000750540917005609175058AE190E00E947F
:105980007313409171056091760584E090E00E9468
:105990007313409172056091770586E190E00E9453
:1059A0007313409173056091780587E090E00E9441
:1059B000731385E0E5E7F5E0A0E7B5E001900D920F
:1059C0008A95E1F7511409F415C88091E00390918C
:1059D000E10320917905211114C08F35914008F41D
:1059E00009C881EE0E9406133092790503C821E0B0
:1059F000823E910508F420E030E0ADCF0E946A05B8
:105A0000B8CF8F35914010F00C94FA2481EE0E94AB
:105A10004613109279050C94FA2480918F01811518
:105A200009F46DC8B0E1B9BDE2E1E9BD09B400FE19
:105A3000FDCF8091D8008F7D8093D8008091E000C9
:105A400082608093E0008091E00081FDFCCF0E94A5
:105A50001D1055C878941F921FB61F9211248F9362
:105A60009F93AF93BF9380917B0190917C01A09114
:105A70007D01B0917E010196A11DB11D80937B0136
:105A800090937C01A0937D01B0937E01BF91AF9173
:105A90009F918F911F901FBE1F9018951F920F927C
:105AA0000FB60F9211242F933F934F935F936F93F1
:105AB0007F938F939F93AF93BF93EF93FF938091C7
:105AC000E10082FF09C08091E20082FF05C0809161
:105AD000E1008B7F8093E1008091DA0080FF24C099
:105AE0008091D80080FF20C08091DA008E7F809363
:105AF000DA008091D90080FFA9C080E189BD82E1F0
:105B000089BD09B400FEFDCF81E08093D903809167
:105B10006A01811109C00E945B0A0E94FE0A8091FD
:105B2000E20084608093E2008091E10080FF1AC06F
:105B30008091E20080FF16C08091E2008E7F80930A
:105B4000E2008091E20080618093E2008091D800C1
:105B500080628093D80019BC85E08093D90383E0EC
:105B6000809305018091E10084FF2FC08091E200C5
:105B700084FF2BC080E189BD82E189BD09B400FEAC
:105B8000FDCF8091D8008F7D8093D8008091E10077
:105B90008F7E8093E1008091E2008F7E8093E2000F
:105BA0008091E20081608093E2008091690181151B
:105BB00009F452C084E08093D9038091D9038430E2
:105BC00009F052C082E0809305018091E10083FFDB
:105BD0002CC08091E20083FF28C08091E100877F84
:105BE0008093E10082E08093D90310926901809153
:105BF000E1008E7F8093E1008091E2008E7F8093B0
:105C0000E2008091E20080618093E20042E060E087
:105C100080E00E94CE0A8091F00088608093F000BE
:105C200081E08093050180930401FF91EF91BF9182
:105C3000AF919F918F917F916F915F914F913F9124
:105C40002F910F900FBE0F901F90189519BC1092B6
:105C5000D90310926A0168CF8091E30087FF02C0E8
:105C600083E0A9CF81E0A7CF81E0ADCF1F920F9253
:105C70000FB60F921124EF92FF920F931F932F9361
:105C80003F934F935F936F937F938F939F93AF93C4
:105C9000BF93CF93EF93FF9309EE10E0F80180815B
:105CA000C091EC008F70C795CC27C795C82B108288
:105CB00080EFE82EF12CF7018081877F8083789434
:105CC0000E943E10F8011082F70180818860808375
:105CD000CF70F801C083FF91EF91CF91BF91AF9149
:105CE0009F918F917F916F915F914F913F912F91F4
:105CF0001F910F91FF90EF900F900FBE0F901F908C
:105D00001895803F09F188F4843901F140F4853316
:105D1000F9F08633F9F0843339F583E20895863952
:105D2000D9F0873909F582E20895853FB9F030F45A
:105D3000813FB1F0843FC1F484E00895863F91F043
:105D4000873F91F487E0089580E0089580E2089508
:105D500084E2089585E2089581E2089585E008953A
:105D600081E0089586E008958FE1089596E8909384
:105D70007A00982F9072906890937B008F71909129
:105D80001A01892B80937C0080917A008064809333
:105D90007A0080917A0086FDFCCF80917800209176
:105DA000790090917A009F7790937A00922F0895CE
:105DB000A8DFDCCFFF920F931F93CF93DF93182FB1
:105DC000EB011092BC0084EA8093BC000E94BB0FE0
:105DD000082FF92E8091BC0087FF28C08091B90060
:105DE000887F883029F08091B900887F803199F5CB
:105DF0001093BB0084E88093BC000E94BB0F182F57
:105E0000092F8091BC0087FF1EC02091B900287F18
:105E100080E090E0283199F081E090E0203411F4A6
:105E200080E090E091958195910909C0802F9F2D88
:105E30000E942815C817D90768F68EEF9FEFCDB7D7
:105E4000DEB7E5E030C4812F902F0E942815C817D7
:105E5000D907B8F6F2CF8FEF9FEFF1CF1092B900CC
:105E60008CE08093B80008950F931F93CF93DF9336
:105E7000EB018093BB0084E88093BC000E94BB0FC1
:105E8000182F092F8091BC0087FF11C02091B90005
:105E9000287F81E090E0283211F480E090E0919535
:105EA00081959109DF91CF911F910F910895CF3F77
:105EB000DC0741F3812F902F0E942815C817D907BE
:105EC00008F78EEF9FEFEECFA0E0B0E0E9E6FFE24B
:105ED000C6C3782EB62EA72E6A0189010E94BB0F79
:105EE0004C010431110508F10F3F100711F1C801F1
:105EF00064E170E09BD3F62EE72E6F2D7E2D872D6B
:105F000059DFEC01892BC1F4EB2CFA2CCE0CDF1CF1
:105F1000EC14FD0411F02097C9F084E98093BC00D3
:105F2000CE01CDB7DEB7EDE0B6C3FF24F394E12C8C
:105F3000E4CF85E0F82EFBCF0F3F1007F1F2C4014C
:105F40000E94281508171907C0F6DECFB801F7011F
:105F500081917F0189DFEC01DBCFA0E0B0E0E2EBD3
:105F6000FFE27DC3782EB62EA72E6A0189010E941A
:105F7000BB0F4C010431110508F10F3F100711F15F
:105F8000C80164E170E052D3F62EE72E6F2D7E2D0E
:105F9000872D10DFEC01892BC1F4EB2CFA2CCE0CF1
:105FA000DF1CEC14FD0411F02097C9F084E9809304
:105FB000BC00CE01CDB7DEB7EDE06DC3FF24F39496
:105FC000E12CE4CF85E0F82EFBCF0F3F1007F1F274
:105FD000C4010E94281508171907C0F6DECFF70183
:105FE0008491B80141DFEC01FFEFEF1AFF0AD9CF2E
:105FF000A0E0B0E0EDEFFFE231C3682E962E5A012B
:10600000690178010E94BB0F782E892E0431110599
:1060100018F10F3F100719F1C80164E170E006D3D1
:10602000162F072F612F702F862DC4DEEC01892BD0
:10603000C1F0FFEFEF16FF06A9F3872D982D0E9400
:106040002815E816F90670F784E98093BC00CE01A4
:10605000CDB7DEB7EEE01EC311E000E0E3CF15E000
:10606000FCCFB701892D00DFEC018501CA0CDB1CD8
:106070000C151D0549F3209739F7B701F8018191F7
:106080008F01F2DEEC01F4CFF5D058F080E891E01A
:1060900009F49EEFF6D028F040E851E059F45EEFA5
:1060A00009C0C0C028C1E92FE07803D168F3092EE8
:1060B000052AC1F3261737074807590738F00E2E6F
:1060C00007F8E02569F0E025E0640AC0EF6307F80F
:1060D000009407FADB01B9019D01DC01CA01AD01A1
:1060E000EF9341D0D5D00AD05F91552331F02BEDFD
:1060F0003FE049E450FD49ECB3C10895DF93DD274B
:10610000B92FBF7740E85FE31616170648075B070D
:1061100010F4D92FF7D09F938F937F936F939CD1D7
:10612000EEEAF8E682D0B4D02F913F914F915F9183
:10613000FAD0DD2349F09058A2EA2AED3FE049EC7D
:106140005FE3D0785D279DD1DF91A2C09AD040F067
:1061500091D030F021F45F3F19F05EC05111CCC0F6
:1061600061C0A7D098F39923C9F35523B1F3951BC8
:10617000550BBB27AA2762177307840738F09F5F68
:106180005F4F220F331F441FAA1FA9F333D00E2ED7
:106190003AF0E0E830D091505040E695001CCAF744
:1061A00029D0FE2F27D0660F771F881FBB1F261709
:1061B00037074807AB07B0E809F0BB0B802DBF01DC
:1061C000FF2793585F4F2AF09E3F510568F024C087
:1061D00093C05F3FECF3983EDCF386957795679527
:1061E000B795F7959F5FC9F7880F911D969587958D
:1061F00097F90895E1E0660F771F881FBB1F6217AC
:1062000073078407BA0720F0621B730B840BBA0B69
:10621000EE1F88F7E095089597F99F6780E870E092
:1062200060E008959FEF80EC0895DF93CF931F9374
:106230000F93FF92EF92DF927B018C01689405C06F
:10624000DA2EEF0170D0FE01E894A59125913591E9
:1062500045915591AEF3EF0114D1FE019701A801CC
:10626000DA9479F7DF90EF90FF900F911F91CF9123
:10627000DF91089500240A941616170618060906D9
:10628000089500240A9412161306140605060895AC
:10629000092E0394000C11F4882352F0BB0F40F434
:1062A000BF2B11F460FF04C06F5F7F4F8F4F9F4F74
:1062B000089557FD9058440F551F59F05F3F71F0F6
:1062C0004795880F97FB991F61F09F3F79F087955D
:1062D0000895121613061406551FF2CF4695F1DFE6
:1062E00008C0161617061806991FF1CF8695710576
:1062F000610508940895E894BB2766277727CB01AA
:1063000097F908959B01AC0160E070E080E89FE39D
:106310000BC1B0DF28F0B5DF18F0952309F07CCF72
:1063200081CF1124E9CFC5DFA0F3959FD1F3950F5D
:1063300050E0551F629FF001729FBB27F00DB11D09
:10634000639FAA27F00DB11DAA1F649F6627B00D99
:10635000A11D661F829F2227B00DA11D621F739F82
:10636000B00DA11D621F839FA00D611D221F749F90
:106370003327A00D611D231F849F600D211D822FD7
:10638000762F6A2F11249F5750408AF0E1F088231E
:106390004AF0EE0FFF1FBB1F661F771F881F91502B
:1063A0005040A9F79E3F510570F036CFA5CF5F3F13
:1063B000ECF3983EDCF3869577956795B795F7955E
:1063C000E7959F5FC1F7FE2B880F911D96958795E6
:1063D00097F9089511F40EF425CFA8C072DFD0F319
:1063E0009923D9F3CEF39F57550B87FFADD00024E7
:1063F000A0E640EA900180585695979528F4805C75
:10640000660F771F881F20F026173707480730F4DC
:10641000621B730B840B202931294A2BA6951794F4
:106420000794202531254A2758F7660F771F881FC4
:1064300020F026173707480730F4620B730B840BE4
:10644000200D311D411DA09581F7B901842F915870
:10645000880F9695879508959B01AC017CC0505894
:10646000BB27AA270ED014CF05DF30F00ADF20F0BB
:1064700031F49F3F11F41EF4D5CE0EF4E095E7FB06
:10648000CBCEE92F16DF80F3BA17620773078407B4
:10649000950718F071F49EF52ECF0EF4E0950B2EB3
:1064A000BA2FA02D0B01B90190010C01CA01A00166
:1064B0001124FF27591B99F0593F50F4503E68F1C1
:1064C0001A16F040A22F232F342F4427585FF3CF02
:1064D000469537952795A795F0405395C9F77EF4D3
:1064E0001F16BA0B620B730B840BBAF09150A1F01C
:1064F000FF0FBB1F661F771F881FC2F70EC0BA0FA2
:10650000621F731F841F48F4879577956795B79529
:10651000F7959E3F08F0B3CF9395880F08F0992721
:10652000EE0F9795879508951CDEB2CE9F3F31F010
:10653000915020F4879577956795B795880F911DB1
:106540009695879597F9089591505040660F771F5B
:10655000881FD2F70895E7DE9BCEB3DE88F09F5701
:1065600090F0B92F9927B751A0F0D1F0660F771F9F
:10657000881F991F1AF0BA95C9F712C0B13081F07F
:10658000BADEB1E00895B7CE672F782F8827B85FBD
:1065900039F0B93FCCF3869577956795B395D9F7E0
:1065A0003EF490958095709561957F4F8F4F9F4FEA
:1065B0000895E89409C097FB3EF4909580957095F6
:1065C00061957F4F8F4F9F4F9923A9F0F92F96E93F
:1065D000BB279395F695879577956795B795F111B4
:1065E000F8CFFAF4BB0F11F460FF1BC06F5F7F4F51
:1065F0008F4F9F4F16C0882311F096E911C0772363
:1066000021F09EE8872F762F05C0662371F096E86B
:10661000862F70E060E02AF09A95660F771F881F3A
:10662000DAF7880F9695879597F90895AA1BBB1BF3
:1066300051E107C0AA1FBB1FA617B70710F0A61B82
:10664000B70B881F991F5A95A9F780959095BC01A3
:10665000CD0108952F923F924F925F926F927F9259
:106660008F929F92AF92BF92CF92DF92EF92FF9262
:106670000F931F93CF93DF93CDB7DEB7CA1BDB0B0E
:106680000FB6F894DEBF0FBECDBF09942A883988B3
:1066900048885F846E847D848C849B84AA84B984BA
:1066A000C884DF80EE80FD800C811B81AA81B981C6
:1066B000CE0FD11D0FB6F894DEBF0FBECDBFED01DA
:1066C0000895992778E0880F991F961708F0961B70
:1066D000881F7A95C9F780950895A1E21A2EAA1B02
:1066E000BB1BFD010DC0AA1FBB1FEE1FFF1FA21782
:1066F000B307E407F50720F0A21BB30BE40BF50B7F
:10670000661F771F881F991F1A9469F76095709507
:10671000809590959B01AC01BD01CF010895052E98
:1067200097FB16F400940FD057FD05D0D6DF07FC79
:1067300002D046F408C050954095309521953F4FC2
:106740004F4F5F4F089590958095709561957F4F5D
:106750008F4F9F4F0895EE0FFF1F0590F491E02D8E
:106760000994692796276927782787277827089526
:106770000FD0A59F900DB49F900DA49F800D911DEB
:1067800011240895B7FFF4CFF3DF821B930B089514
:10679000A29FB001B39FC001A39F700D811D112462
:1067A000911DB29F700D811D1124911D0895FB0153
:1067B000DC0102C005900D9241505040D8F7089579
:1067C000FB01DC0104C08D910190801921F441503E
:1067D0005040C8F7881B990B0895DC0101C06D93E8
:1067E00041505040E0F70895DC01CB01FC01F999DC
:1067F000FECF06C0F2BDE1BDF89A319600B40D920D
:1068000041505040B8F70895F999FECF92BD81BD2F
:10681000F89A992780B50895A8E1B0E042E050E0E9
:10682000E5CFDC01A40FB51F4150504040F0CB0133
:10683000840F951F2E9105D041505040D8F70895F0
:10684000262FF999FECF92BD81BDF89A019700B429
:10685000021639F01FBA20BD0FB6F894FA9AF99AC9
:106860000FBE08950396272FECDFEADF252FE9DF1F
:10687000242FE7CF0196272FE4DFE2CFDC01CB0105
:1068800002C02D9105D041505040D8F70895262FD1
:10689000F999FECF1FBA92BD81BD20BD0FB6F89405
:1068A000FA9AF99A0FBE01960895F894FFCF084A14
:1068B000D73B3BCE016E84BCBFFDC12F3D6C743114
:1068C0009ABD56833DDA3D00C77F11BED9E4BB4C6B
:1068D0003E916BAAAABE000000803F001A11401131
:1068E0004611401146119811B9114611C012CD122E
:1068F000151B7D1B1D1BE71AEB1A211BEF1A251B0D
:10690000311BFB1A761BFF1A351B031B391B5E1B41
:10691000071B3D1B651B0D1B431B4B1BF31A291B40
:10692000F71A2D1B111B471B551B6E1B741BE11AFD
:10693000191B841BB31AB91AA61AAD1ABF1AC51AA5
:10694000CB1A252B3C2B432B82298229772B892B91
:106950009C2BDB2BE02B822982298229E92B6F29B2
:106960007329A029AE29B929C4296C296C296C295D
:106970006C29102BC729CA29CE29FA29382A3B2A83
:046980003D2A712A11
:10698400FF00000001004E09B90BAF09B009B109BD
:10699400B00B0021007F2200030140776173640083
:1069A4003E15C132C3DECD830044221CEA00C80078
:1069B400AC0034074D076D073133323635346694F5
:0C69C40097C6F700081018181008000013
:00000001FF
